:020000040800F2
:10500000A0300020D5500008CDA30008C9960008A4
:105010000000000000000000000000000000000090
:1050200000000000000000000000000029AB0008A4
:105030000000000000000000CFA3000855B10008E8
:10504000E7500008E7500008E7500008E750000864
:10505000E7500008E7610008E7500008F761000822
:1050600000000000E7500008E7500008E750000883
:10507000E75000084D9A0008E7500008E750000884
:10508000E7500008E7500008E75000080000000063
:10509000E7500008E7500008E7500008E750000814
:1050A000E7500008E7500008E750000809BF000873
:1050B00019BF00088D9B00080000000000000000E0
:1050C0000348854600F0D6FC004800478DCE000816
:1050D000A03000200448804704480047FEE7FEE770
:1050E000FEE7FEE7FEE7FEE715B20008C150000844
:1050F00030B50B46014600202022012409E00D4670
:10510000D5409D4205D31D469540491B25469540F7
:1051100040191546521E002DF1DC30BDF0B51FB40C
:105120000646002082B005464024019100901BE015
:10513000019922460F46304600F080FB049A059BF9
:10514000801A994110D310461946224600F066FB9A
:10515000361A8F410197224601200021009F00F05E
:105160005DFB38184D4100902046641E0028DFDCAE
:10517000019B00982946324607B0F0BD03460B4319
:105180009B0703D009E008C9121F08C0042AFAD2FD
:1051900003E00B780370401C491C521EF9D2704783
:1051A000D2B201E00270401C491EFBD270470022BF
:1051B000F6E710B513460A4604461946FFF7F0FF16
:1051C000204610BD30B505462A460B4610781C789F
:1051D000521C5B1C002801D0A042F7D0002C03D049
:1051E000002802D06D1CEFE7284630BD421C017834
:1051F000401C0029FBD1801A704730B504460020BE
:10520000034600E05B1C934203D2E05CCD5C401B94
:10521000F8D030BD70B5064607F076F9046805464B
:105220000A220021304600F02DFB2C6070BDF8B53D
:1052300002464A40D40F42004B0052085B089A4293
:1052400002D20246084611464A0023D0C30D4A0046
:10525000DDB2120EAD1A202D35DA49020126490AB7
:10526000F6058A19002C00D0524220214F1B11460E
:10527000B9402A411018C20D9A4221D0002C17D0F3
:10528000012D08DCDA05801AD20F8019D207DBB2B3
:1052900000F038FBF8BDDA05801A012340001B0638
:1052A000C01880185A428018CA0F1043490007E0FE
:1052B0004908C2071143DA05801A8019400880188E
:1052C00000F018FBF8BD61000122511A001BF7E73E
:1052D0000122D2075140AAE70122D2075040A6E797
:1052E000024670B54A40D30FDB0740002DD04A007C
:1052F0002AD0010E140E000212020919400A520AA5
:105300008418E50104465443000A120A2E0450434F
:10531000A4194219200CC543AA18120C0125AD038B
:10532000521C521912047F39240400D0521C10431D
:1053300001D44000491EC2B20C06C0092018401C0E
:105340004008802A02D003E0002070BD40084000E1
:10535000002900DA0020184370BD70B502464A40AB
:10536000D50F40004A00ED0740085208002814D02D
:10537000002A12D0C40DD30D41020120C0055202F3
:10538000490A520AE41A091812187D34914201D3CD
:10539000641C00E04900002C01DA002070BD0023ED
:1053A000914201D3891A0343400849000028F7D1EC
:1053B00000290AD0914202D10121C90705E091429A
:1053C00001D2012101E00121C943E005C0184019C3
:1053D00000F090FA70BD420005D04200120E524219
:1053E0008A4201DB00207047C90508187047000099
:1053F000F0B507460846584087B0C00F04904800F3
:105400000E46590040084908BC1A884105D2384662
:1054100031461E4617460B460246580040081043C8
:105420004CD0300D039040055900400D490D0590BA
:10543000401A0290402872DA18030121000B090576
:105440000843019004980092002805D00199524227
:105450000020884100920190029840210A1A019987
:10546000009800F0DBF905460C466B4607CB00F0D0
:10547000F6F9C0197141039A0E0D0023D717564053
:105480001A467A40164344D0049A002A2DD0029A34
:10549000012A039A15DC1205C01A9141012636052E
:1054A000001C7141D20F059ED20700930192029613
:1054B0002A46234600F06CFA07B0F0BD3846314664
:1054C000FAE71605224A0F46B218C01AB741012161
:1054D0000905001C4F4100187F41114618187941F9
:1054E000E20F10436D19644113E0E2076D081543A4
:1054F0006408C2071443039A01261205C01A914199
:105500003605001C7141CE07400830434908C018D9
:1055100051412A46234600F02EFACDE7FFE70498D2
:1055200001224000C117121A00238B410498314612
:10553000C417381AA141EEE730B40124E4076340F0
:1055400030BC55E730B40124E407614030BC4FE77C
:105550000000E0FFF0B51FB488B00B990998002453
:1055600048400999C00F490049080991C0070B99A3
:105570000090490049080B9109990898A6460843EC
:105580001CD00B990A98084318D0099801244000B0
:10559000420D4800410D099824050003000B2043EB
:1055A00009900B980003000B20430B9050181C49E6
:1055B0004018002201901446104605E000200146E4
:1055C0000DB0F0BD032801DA034600E003239C463A
:1055D000C11A0AAE0AE05F0008ADED5B4F00F75B51
:1055E0007D430027AA187C41491C5B1E6145F2DD02
:1055F000410004AB5A522104120C0A43240C401CF3
:105600000828DFDB01980290009970460191009014
:10561000059B049A0799069800F0BAF9D0E70000B4
:105620000DFCFFFFF0B50C465C4085B0E40FE407CD
:1056300003944C0000266408590094464908024629
:105640000296224321D062460A431ED06200570DC3
:105650004A000E032303550D012402462C4924055C
:10566000781B1B0B360B40182343264361460090E2
:105670001C46501AB44103D30098401C009002E02D
:10568000921800985B41002803DA0020014605B01B
:10569000F0BD0020012109050746864611E0644659
:1056A0001D46141BB54106D36546521BB3417446D3
:1056B00007430C43A646CD074008490828439218E3
:1056C0005B4105460D43EAD11046184313D06046AE
:1056D000194650407140084306D06046101AB34145
:1056E00006D20122002306E000220123DB0702E0AC
:1056F0000122D2435310009874460105381C6141C1
:10570000029C039D0019694100F035F9BFE70000D4
:10571000FD0300000EB505490291002100910A46E3
:105720000B46019100F034F903B000BD33040000D2
:10573000410040020122400AD205090E80187F294B
:1057400001DA00207047962903DC9622511AC840DE
:1057500070479639884070474A0009030123090BB6
:105760001B051943094B10B5520D9A4201DA00206E
:1057700010BD064B34339A4203DC9A1A00F05EF8EF
:1057800010BD03495118884010BD0000FF03000000
:10579000CDFBFFFFC20FD207400040080BD0C10D68
:1057A0000723DB01C91840020905400A1143C2085A
:1057B00040071143704700200146704710B500298B
:1057C00004DB0124E40740428C412146002B04DB2A
:1057D0001C460123DB075242A341994200D190426B
:1057E00010BD0000CB0FDB07490010B54908024689
:1057F0000A4307D00A0D07240903E401090B121B11
:10580000002A01DC002010BDC900440F0C43C10078
:10581000E018D205801800F06DF810BD10B5202AF0
:1058200004DB0146203A9140002010BD9140202326
:105830009C1A0346E3401943904010BD10B5202A3E
:1058400004DB0846203AD040002110BD0B46D3406F
:10585000D0402024A21A91400843194610BD10B52B
:10586000202A06DBCB170846203A1041C1170B430C
:1058700006E00B461341D0402024A21A9140084371
:10588000194610BDF7B5009C0F4600262578641C0C
:10589000002D05D000F000F90068405DC007F5D18B
:1058A0002B2D02D02D2D18D0641E39462046029A89
:1058B00000F0F6F8002F04D03968A14201D1009918
:1058C00039607105022400290BDA4042002803DD0B
:1058D00006F01AFE0460A007FEBD01208002064308
:1058E000E3E70028F8DA06F00FFE04600048FEBD8A
:1058F000FFFFFF7F002904DA401C490001D1400866
:105900004000704770B40024050C05D11024000439
:1059100002D1002921D01124050E01D10002083442
:10592000050F01D10001241D850F01D18000A41CA9
:10593000002801DB4000641C002908D020252E1B14
:105940000D46F540A14000D001212943084301063E
:105950001B1B000ADB1D02D5002070BC7047DB0555
:10596000181880180029F8DA401C4900F5D170BCDD
:1059700040084000704710B5002B08DA0024401C96
:10598000614192185B411A4301D14008400010BDAB
:10599000F0B51FB482B005460C0003D0084606F0EF
:1059A00067FD02E006F064FD2030024600902146CB
:1059B0002846FFF733FF049B059A04460F46184319
:1059C0001143084314D0184610431BD000984021BF
:1059D0000A1A18460599FFF731FF05460E46009A48
:1059E00005990498FFF71AFF084305D0012004E049
:1059F0002046394607B0F0BD0020C11705430E43CD
:105A00002C43374300990E986305401A7905E40A40
:105A100000220C43FD0A0A3002D500200146E9E7C6
:105A20000105101969410C9C0D9D00196941FFF792
:105A3000A2FFDFE74A0009030123090B1B051943F5
:105A40000A4B10B5520D9A4202DA0020014610BDF1
:105A5000064B34339A4203DC9A1AFFF7EFFE10BD6F
:105A6000034BD218FFF7DAFE10BD0000FF03000061
:105A7000CDFBFFFF064C0125064E05E0E36807CC91
:105A80002B430C3C98471034B442F7D3FFF71CFB70
:105A9000B0D40008D0D400080048704710D30008E4
:105AA000F7B582B0029C00272078641C1546019748
:105AB000302802D0002D15D015E020780127641C75
:105AC000782804D0582802D0002D09D00BE0002DF2
:105AD00001D0102D07D1002710252078641C02E08A
:105AE000082500E00A250026009610E0009901270D
:105AF00069430818020C294680B2714300908E1841
:105B00003804864201D3012001902078641C294684
:105B100000F019F80028E9DA0398002805D0002FD2
:105B200001D0641E00E0029C04600198002806D0A9
:105B300006F0EAFC02210160C81E05B0F0BD009924
:105B400030040843F9E73A2800D2303820230246CF
:105B50009A43412A01D310463738884201D30020A6
:105B6000C043704770B58C180578401C6B075B0FFD
:105B700001D10378401C2A1106D10278401C03E0B1
:105B800006780E70401C491C5B1EF9D12B0705D40A
:105B90000023521E0DD40B70491CFAE70378401CF9
:105BA000CB1A921C03E01D780D70491C5B1C521E21
:105BB000F9D5A142D8D3002070BD70B50446206845
:105BC0008168490727D5816810254907002905DA2A
:105BD0008168890702D481682943816001F07CFAD9
:105BE000064620688068400715D501F075FA801BCD
:105BF0000A280CD920688068400708D5606D2843C2
:105C00006065A06D01210843A065012070BD20687A
:105C100080684007E9D4002070BD000038B5044614
:105C2000094808490068FFF763FA6043009000984C
:105C3000002805D00098401E009000980028F9D157
:105C400038BD000040420F0008010020F8B50446AE
:105C5000206881688907890F012934D10168C90743
:105C600031D081680522114010250126012907D075
:105C7000606D28436065A06D3043A0650120F8BDCC
:105C8000816802221143816021680320086001F0CD
:105C900023FA074620688068C00714D001F01CFA78
:105CA000C01B0A280BD920688068C00707D0606D28
:105CB00028436065A06D3043A0650120F8BD2068D1
:105CC0008068C007EAD10020F8BD0000F8B504469E
:105CD000206881688907890F012902D10168C907F5
:105CE00033D181681A4A102611400125002907D0B6
:105CF000606D30436065A06D2843A0650120F8BD4C
:105D00008168294381600120FFF788FF01F0E4F9F1
:105D1000074620680068C043C00716D001F0DCF9D0
:105D2000C01B0A280CD920680068C043C00707D0F0
:105D3000606D30436065A06D2843A0650120F8BD0B
:105D400020680068C043C007E8D10020F8BD00000B
:105D50001700008010B50E4800F0BEFF00F0C0F93B
:105D600005F05CF800F02EFB0A480B49808C0860B7
:105D70000A4C0020A06000F04FF8094800F09CFC9D
:105D800000F0C6F8207003F041FF002010BD0000B5
:105D9000B80B000074060020280000203800002006
:105DA000B963000870B503F0E1F903F093FD00F06A
:105DB0002BFC03F06DFF1448144C00786178084305
:105DC00001D104F005F903F04BFF012801D103F0E4
:105DD00085FD0E4810308188006801F06FF90128B8
:105DE00005D00B480025007800280AD007E00948B4
:105DF00001250078C00704D000F03CF9A570002010
:105E000070BD00F019F9F9E73000002038000020DB
:105E1000990000202800002010B5012007F08EF81E
:105E20000A4C1328A0700AD0E01C03F0C3FDE078F0
:105E3000A070332806D006490020C88710BD07F09F
:105E4000B5F810BD03F088FD10BD0000D80000209B
:105E50007406002010B500F003F8002010BD00000B
:105E600070B50524FF22240701322146012004F0E9
:105E7000C7FA1749002006F04BF91649022006F030
:105E800047F91549012006F043F9144D0122920308
:105E90002946002003F0EEFE04222946012003F0EB
:105EA000E9FE012212032946022003F0E3FE10223C
:105EB0002146002000F0A0FB0021094800F0FCF87A
:105EC0000122D2022146012000F070F8002070BDAE
:105ED000CC0400205405002044040020000400509D
:105EE0003406002010B50024084800F023FE611E8F
:105EF000064800F0B7FD002803D1044800F08CFCF0
:105F00000446024800F046FE204610BDB8030020BB
:105F100070B5002400F026F80D4E0546B04215DBA2
:105F200000200C4A0C4B0146FFF748FC01D26424C8
:105F30000CE031462846FFF7CBF90849FFF70DFA88
:105F40000749FFF7CDF9FFF7F3FB0446204670BD84
:105F500033335340CDCCCCCCCCCC10406666663FBE
:105F60000000C84210B500F017F8642000F0B4FE3D
:105F7000FFF7B8FF00F048F8044600F003F82046A9
:105F800010BD000010B5034801228189806801F02E
:105F90009CF810BDDC11002010B503480022818957
:105FA000806801F092F810BDDC110020022802D3B5
:105FB0000020C0437047C3000248C15018188280B7
:105FC00000207047DC11002010B50C4C206B00281D
:105FD00012D16169A06A401A3C280DD308490020FB
:105FE0000870FFF795FFC1B206486429017001D916
:105FF00064210170A06A606110BD000000000020F3
:10600000390000203800002010B5FFF783FB002284
:10601000064BFFF707FB064A064BFFF79BFAFFF715
:10602000E1FB0121FFF7D7F910BD000000FEAF40F2
:106030006666666666660A4010B50D4C002320460B
:1060400000686168026800290BD004290BD0082978
:106050000BD0136402F052FA206802F0C1F800205D
:1060600010BD5363F6E79363F4E7D363F2E70000F0
:106070008000002010B50F4C206802F081F803CC9E
:10608000083C02F0F1F961683C20002908D004299D
:106090000AD00829216809680AD00864002010BDC8
:1060A000216809684863F9E7216809688863F5E7AA
:1060B000C863F3E780000020014A03C20020704754
:1060C0008000002010B500231A4603E0845CE3182A
:1060D0009BB2521C8A42F9D3D84380B210BD000053
:1060E00000B587B0012168464170022101700D485A
:1060F0000190C801029080000490402005906946FC
:10610000002005F051FF0748074920380161074981
:10611000C1610749816107494161074802F01CFFDD
:1061200007B000BDDC100020496100083D61000897
:1061300079610008876100083C0B002010B501461A
:10614000002005F0F1FE10BD0FB400B5FFB082B025
:10615000012183AB49026846829A06F073F96846CA
:10616000FFF744F802466946002006F035F87FB094
:1061700002B008BC04B0184701B5012269460020EE
:1061800006F02AF808BD10B50446FFF72FF80246BE
:106190002146002006F020F810BD30B4446C1C25C8
:1061A0002C400125A540046C656004686360836829
:1061B000102B05D0036899600068C26030BC70473E
:1061C00003689A600068C16030BC704708B503E09E
:1061D0006846007806F0AEF86946002005F0A4FE97
:1061E0000028F5D008BD10B5012000F0A1FE022066
:1061F00000F09EFE10BD10B5202000F099FE80201A
:1062000000F096FE10BD000010B4084900234B6159
:1062100007494A684C1522434A604A6808242243C9
:106220004A60C009C001036010BC70478829002083
:10623000002002407FB500250C460646039500F07D
:10624000C9FDE009029003A901960095684600F097
:1062500055FD002804D000F091FD002004B070BD71
:1062600000F08CFD0120F9E710B5002302E0C45CCA
:10627000CC545B1C9342FAD310BD000010B4002034
:10628000204A9169CB05204904D548690223184367
:106290004861901593699B0505D54B6901242343FB
:1062A0004B616302184393695B0505D54B6908246C
:1062B00023434B61E301184393691B0505D54B69E3
:1062C000042423434B616302184393699B0405D55F
:1062D0004B69102423434B616302184393699B036A
:1062E00004D54C6920231C434C6118439369DB039C
:1062F00005D54B69402423434B61A10208439061BB
:1063000010BC7047002002408829002070B5044668
:1063100000F0E2FE0546194EB069C0070DD0601CC2
:1063200008D0002C04D000F0D7FE401BA04201D9B9
:10633000032070BDB069C007F1D1B069800701D5F5
:106340000220B061B069C00511D4B06980050ED4D7
:10635000B06940050BD4B069000508D4B069800469
:1063600005D4B069800302D4B069C00303D5FFF738
:1063700085FF012070BD002070BD0000002002409C
:10638000F8B51746002605460C4600F023FD09E047
:1063900029460220226800F0FFFC002804D1241DB9
:1063A0002D1D361DBE42F3D300F0E8FCBE4201D2E3
:1063B0000020F8BD0120F8BD01490220C8707047D7
:1063C0003800002000B587B00120694648700220DF
:1063D00008700C490191410202910B49039105217A
:1063E000490204910590694605F0DEFD88210748C1
:1063F00002F066FF052001221021000700F065FE73
:1064000007B000BD6C1200206C1600207C2000201C
:10641000F0B593B00E460546282108A8FEF7C7FE42
:1064200003AA00922846314601AB4FA202F079FF41
:106430000027FF4302281AD10499039802F061FF54
:10644000C2B201980178012003E0019B1B5C594016
:10645000401C029B8342F8D8914208D1002406AB2D
:1064600044A23146284602F05CFF0F2802D038468D
:1064700013B0F0BDA819801E0470447049482B4623
:10648000027849484188049202910394059447494F
:106490008088097801910090FF2145A201314B4885
:1064A00003F032F8074680214948FEF780FE3A465D
:1064B00046494748FEF762FE464D474EAF70069884
:1064C00039460078302841482AD002F035FD686806
:1064D000002846D041A002F00FFD6B683A463B49C8
:1064E000002098476878002803D0FF2030606C7047
:1064F00002E001203460687037483C4D3C4E3D4F0F
:1065000002682B683168386804F04CFB642000F0A6
:10651000E3FB3148224604602B68316838681EE08E
:1065200002F00AFD6878002804D0FF2000023060E5
:106530006C7002E00120346068702C4D2C4F2D48A7
:106540002B6832683968006804F02CFB642000F086
:10655000C3FB3460274822462B683968006804F082
:1065600021FB002084E700002425702A25700D0AF5
:106570000000000024252A2C252A2C252A2C252A37
:106580002C252A2C252A2C25702C252A2C252A2C32
:10659000252A2C252A2C252A2C252A2C252A2C256F
:1065A0002A2A00003A00002074060020380000204B
:1065B00025732C25582C253032782C25782C2564F1
:1065C0002C25782C2564250D0A00000004210020CC
:1065D000EC1100208C0000201C0000204C4F524188
:1065E0002046414641464146410D0A001800002020
:1065F0002000002024000020C3000248C1501818C9
:10660000828070476C20002008B500206946087021
:1066100003E06846007800F013F86946022005F0B0
:1066200083FC0028F5D008BD0149002008707047A0
:106630008C00002001490120087070478C00002068
:1066400070B51A4D00262C462B78611C8034002B27
:1066500008D022465268022B0CD0032B09D10A28FD
:1066600013D021E0242804D102222A707054012082
:10667000606070BD50546168491C61607E2913D20E
:106680000D28F6D10320287070BD50546068401C5E
:106690006060465406A1681CFEF794FD002803D0F4
:1066A000681C6168FFF7B4FE2E7070BD7C2000206E
:1066B0004747412C00000000014948607047000036
:1066C0008C000020F8B50C4605464035297C012990
:1066D0000DD00121297401688A68520709D5416DDE
:1066E000202211434165002028740120F8BD0220BA
:1066F000F8BD194B6268D8054710184E9A4215D05C
:106700008A6A23685B035B0B1A438A622168490328
:1067100005D5B1680143B1600A20FFF77FFA206810
:10672000800315D5B0683843B06011E08A6A2368E9
:106730005B035B0B9A438A622168490302D5B16807
:106740008143B1602068800302D5B068B843B0606F
:1067500000202874F8BD000001100000002701404F
:1067600070B50446002C0AD0606D022108436065B4
:106770002046FFF722FA0546280002D009E0012052
:1067800070BD2046FFF762FA0546012D01D00120B9
:1067900060650026012D32D0206841681A4A1140F8
:1067A00041602168D0430860206881680122120797
:1067B000914381602068C168144A1140C16020681B
:1067C0000169134A1140016120684169C908C90083
:1067D00041612068016A0F4A1140016220688030DF
:1067E000416BC909C901416320688030416BC90907
:1067F000C9014163204600F0F9F8A665666540349A
:106800002674284670BD000060F7FFFF00023E833B
:1068100002FCFF3F00F000F00068006C70470000D1
:1068200070B50446002C06D0606D26460025403623
:10683000002802D006E0012070BDA5653574204611
:1068400000F0E8F8606DC00603D42068816849074D
:1068500006D5606D1021084360653574012070BD58
:10686000616DFF220132914302221143616581680B
:106870005C4A8907890F012902D10168C9072BD118
:10688000032361689B07994205D05B42994202D07D
:106890005B00994209D1016989008908016120687A
:1068A00001696368194301610CE001698900890885
:1068B000016190680F218904884390609068616845
:1068C000084390602068C16818239943C16020681C
:1068D000C168A3681943C1609068012149068843D3
:1068E00090609068A18E4906084390602068816896
:1068F000C90004D481680122120711438160206815
:10690000C168394A1140C1602069E268022825D077
:1069100000200243204620300178037B49035B00BE
:1069200019430A43216B0A43A16989030A43E169B8
:10693000C9030A432168CB681A43CA60616A0A46E0
:10694000FF3AC23A05D0A26A11432268D3681943BC
:10695000D16042780121012A02D00BE00420D8E75F
:106960000078002823D0606D202210436065A06D60
:106970000843A065E06B012820D020680169C907A1
:1069800003D0016949084900016120684169C908CB
:10699000C900416120684169A26B11434161A5654D
:1069A000606D80088000401C6065002070BD20681C
:1069B000C26801231B041A43C260DBE72068026936
:1069C000FF239B009A43026120680269236CA66C36
:1069D0001A43636C33431A430261206802690A4315
:1069E0000261D2E7002701401902FEFF10B50068DE
:1069F0000649884209D10648416B421591434163DB
:106A000005200221000700F015FA10BD0024014006
:106A10000010024010B586B0044614216846FEF707
:106A2000C6FB0E492068884216D10D48416B4215BD
:106A300011434163C16A01221143C162C06A6946C0
:106A40001040059002200090032001900020029049
:106A50000520000700F078FA06B010BD00240140C0
:106A600000100240F8B504460E46274660694037DC
:106A700008280BD02068C068C00709D0606D2021AD
:106A800008436065002038740120F8BD082500E047
:106A90000C2500F021FB009020680068284219D1E5
:106AA000701C13D0002E05D000F016FB0099401A80
:106AB000B0420BD920680068284207D1606D0421DC
:106AC00008436065002038740320F8BD2068006822
:106AD0002842E5D0606D01214902084360652068C5
:106AE000C16809058A0F0C21002A1BD12022125DE2
:106AF000002A17D10268120714D5826801235207B1
:106B0000002A08DB42688A434260606D1A029043A3
:106B10001843606506E0606D202210436065A06D3B
:106B20001843A065A069002801D1206801600020F9
:106B3000F8BD000070B50446002021688968490747
:106B400023D425464035297C01291CD001212974F4
:106B5000E169012902D02046FFF7B8F8002811D1D9
:106B6000616D0B4A1140FF22013211436165002122
:106B7000A165297422681C21116021688A68042398
:106B80001A438A6070BD022070BD022070BD0000F3
:106B9000FEF1FFFF70B5044625464035287C0128EC
:106BA00007D001262E742046FFF707F8002802D0F0
:106BB0000CE0022070BD2046FFF748F8002805D100
:106BC000616DFF22013291433143616500212974D7
:106BD00070BD30B4014620314A790023022A05D025
:106BE0000422C2630B7130BC012070470268146834
:106BF0000E25AC43146002681468640864001460D5
:106C0000446C1C22144001252A46006CA2404260BC
:106C10004D710B7130BC1846704770B500240146A9
:106C200020314A79022A03D00421C163012418E0EB
:106C3000026813680E25AB431360026813685B0893
:106C40005B001360436C1C22134001252A469A40C6
:106C5000036C5A604D7100220A71816B002900D0CB
:106C60008847204670BDF8B504468C46002520466E
:106C700020300179012909D00126067147790021C8
:106C8000012F05D0017102252846F8BD0220F8BD6C
:106C900002274771E16320680168490849000160E3
:106CA00061462046FFF779FA206B002805D020685E
:106CB00001680E221143016009E020680168042286
:106CC00091430160206801680A2211430160206835
:106CD000016831430160D7E770B5044600F0FCF964
:106CE0000546601C02D004480078241800F0F4F92E
:106CF000401BA042FAD370BDFC000020F8B5054649
:106D00000E461B4F387C012808D0012038741948E2
:106D1000FFF7FCFA0146080002D025E00220F8BD8A
:106D20000020C04330606C68A868C0010019A04210
:106D30001AD92046FFF768FA0E48FFF7E7FA01462E
:106D40000D48426808239A434260426843159A43BB
:106D50004260002901D0346006E08034A8686A6887
:106D6000C0018018A042E4D8002038740846F8BD5D
:106D70008829002050C300000020024005484168D7
:106D80000222114341604168012211434160002009
:106D90007047000000200240F8B50E4617460B4C25
:106DA000207C012808D0012020740948FFF7AEFAA2
:106DB0000025002802D006E00220F8BD656137609A
:106DC0000348FFF7A3FA2574F8BD000088290020C6
:106DD00050C3000012494868C0070DD0EFF310807F
:106DE00072B6104ACA60104ACA6080F310884868B8
:106DF000C00701D001207047486880070DD5EFF328
:106E0000108072B6094A0A61094A0A6180F3108843
:106E10004868800701D501207047002070470000B6
:106E200000200240EFCDAB8905040302BFAE9D8C6C
:106E300016151413F0B50022002961D001239340E8
:106E40009E460B40002B57D095082E4CAD002D19B7
:106E5000AC689607360F0F27B7403C40A446052480
:106E60002407A04201D1002419E0274CA04201D1FF
:106E7000012414E0254CA04201D102240FE0244C4F
:106E8000A04201D103240AE0224CA04201D10424F3
:106E900005E0214CA04201D1052400E00624B440C5
:106EA00064450FD11D4C26689E43266066689E434C
:106EB0006660E6689E43E660A6689E43A660AB688F
:106EC000BB43AB60046855000323AB401C43046024
:106ED000D408A4002418266A5507EF0E0F25BD40DC
:106EE000AE432662C4689C43C46044687546AC43A4
:106EF000446084689C438460521C0B46D3409DD1FF
:106F0000F0BD0000000001400004005000080050E7
:106F1000000C005000100050001C00500004014004
:106F2000202802D101490020086070472C00002071
:106F300010B504494A69024202D04861FFF7F0FFE8
:106F400010BD000000040140F0B400220B68002BCB
:106F50006FD001270B6897403B40002B6AD00C791B
:106F6000A407A40F012C01D0022C10D18568540075
:106F70000326A640B543CE68A6402E4386604468EB
:106F8000BC430D79ED06ED0F9540254345600C7926
:106F9000E443A40708D0C56854000326A640B543BF
:106FA0008E68A6402E43C6600C79A407A40F022C5D
:106FB0000CD1D408A40027183D6A5407E40E0F260C
:106FC000A640B5430E69A6402E433E6205685400B4
:106FD0000326A640B5430E79B607B60FA6402E434A
:106FE00006604C68A403A40F50D02C4C656B01269E
:106FF0003543656395082A4CAD002F19BD68940789
:10700000240F0F26A640B54305263607B04201D10E
:1070100000261BE0234EB04201D1012616E0224E8D
:10702000B04201D1022611E0204EB04203D1032626
:107030000CE030E02AE01E4EB04201D1042605E00B
:107040001C4EB04201D1052600E00626A6402E4384
:10705000BE60194DAC689C434E68F60200D51C43D7
:10706000AC60EC689C434E68B60200D51C43EC60F3
:107070006C689C434E68B60300D51C436C602C685A
:107080009C434E68F60300D51C432C60521C0B68D1
:10709000D34000D05DE7F0BC704700000010024014
:1070A000000001400004005000080050000C005097
:1070B00000100050001C005000040140006908420C
:1070C00001D00120704700207047002A01D0816163
:1070D0007047816270470000014880687047000077
:1070E000FC00002004494A6B01231A434A63034908
:1070F0004A6802434A6070470010024000000140A5
:10710000024881680278891881607047FC0000207D
:1071100010B5002407480168402211430160032094
:1071200000F00AF8002801D0012401E000F084F901
:10713000204610BD0020024070B504460E4D7D2053
:107140002978C000FDF7D4FF01460C480068FDF720
:10715000CFFF00F065FF002801D0012070BD042C96
:1071600007D200222146501E00F08EF96C600020EC
:1071700070BD012070BD0000FC000020080100204F
:107180007047704710B51148114B816A491C8162E4
:10719000C16A491CC16218780021012807D10D4835
:1071A0000268521C0260022A01D3016019700A4869
:1071B0000278012A09D1094B1A78521E1206120EC2
:1071C0001A7002D10170FEF737FF10BD00000020D9
:1071D0007500002058000020990000209800002031
:1071E0007047704770472030807B704710B5044669
:1071F00020680168C943C90708D18168C943C90724
:1072000004D1012141602046FFF7BCFF20680168DE
:10721000C943890708D48168C943890704D4022176
:1072200041602046FFF7ACFF20680168C943490769
:1072300008D48168C943490704D404214160204629
:1072400000F0F8F820680168C943090708D481688C
:10725000C943090704D4082141602046FFF7C0FF55
:1072600020680168C943C90608D48168C943C906B2
:1072700004D4102141602046FFF783FF2068016895
:10728000C943890608D48168C943890604D42021EA
:1072900041602046FFF7A6FF20680168C943490600
:1072A00008D48168C943490604D44021416020467E
:1072B000FFF797FF10BD0000F8B50446002C06D07C
:1072C000606825462035A87B002802D006E0012012
:1072D000F8BD00206873204600F046F80220A8732D
:1072E00020688446C0686168012904D00122A36A2D
:1072F000D205934201D11E229043184B62699A42F3
:1073000001D0174B1840174B1840A368676A266ACC
:107310000B433E431E43A36A1E433043002903D15F
:107320002769E6693E433043012903D00121C9059D
:107330008B4203D12369E1681943084307498A4214
:1073400005D0A1690A43E16901431046084361463B
:10735000C8600120A8730020F8BD0000FFFF0000F6
:107360003F1FFFFFFEF119FF10B500680849884272
:107370000CD10848816BC20411438163002211467D
:107380000D2000F081F80D2000F072F810BD000013
:10739000007C004000100240F8B504461646022268
:1073A000204620300546827321480268C3041A43F0
:1073B00002602068C2689B121A43C260206802699A
:1073C00001273A43026122681020506020688161E1
:1073D0001021204602F0BCFB032822D0216808209F
:1073E0004860206846610821204602F0B1FB03286E
:1073F00019D0204602F032FB2046FFF7F4FE0328A6
:1074000013D020688168394381602068016939435D
:10741000016120680169042211430161AF730020FA
:10742000F8BD0320F8BD0320F8BD0320F8BD00001F
:1074300000040140704700000448416B01221143E1
:107440004163816B02041143816370470010024065
:10745000002809DBC106C90E0120884003490860E5
:10746000BFF34F8FBFF36F8F7047000080E100E0E4
:10747000002805DBC106C90E0120884001490860CB
:107480007047000000E100E08207D30EFF229A401F
:107490008907090E9940002808DB830809489B00EA
:1074A0001818036893430B43036070470007000FED
:1074B0000838830804489B001818C36993430B439A
:1074C000C361704700E400E000ED00E0024801689D
:1074D000821511430160704700700040F0B4164EF1
:1074E000326875152A40154B1B6ADB07DB0F002A33
:1074F00004D0002B02D03468AC4334603468A40854
:10750000A400044334600E4F3C69042004433C61F2
:1075100001290ED040BF20BF20BF396981433961A6
:10752000002A04D0002B02D0306828433060F0BC21
:10753000704730BFF1E700000070004000000140DC
:1075400000ED00E0F8B50446002620785E4D800688
:107550007DD55E48806BC00005D45C48816B020419
:107560001143816301265A480168C90517D4006890
:10757000FF210131084356490860FFF7ADFD07467A
:1075800053480068C0050AD4FFF7A6FDC01B642855
:1075900001D90320F8BD4E480068C005F4D54B4F13
:1075A000386803210905084062681140814208D00B
:1075B0009003800F032804D13868800301D501208F
:1075C000F8BD2869032109040840002824D00A4096
:1075D000824221D0207880061ED5286988432A69F6
:1075E0000121C9040A432A612A698A432A61286160
:1075F000C00511D5FFF770FD0090286980050BD4F8
:10760000FFF76AFD0099411A3248814201D90320EF
:10761000F8BD28698005F3D52078800611D560680B
:107620008103890F032905D13A6809058A43084077
:1076300002433A602869032261681204114008433A
:107640002861012E03D1B96B30078143B9632078DB
:10765000C00705D0E868A168800880000843E8609A
:107660002078800705D5E8680C218843E168084345
:10767000E8602078400706D5E8680321890288433E
:1076800021690843E8602078000706D5E8680321EF
:107690000903884361690843E8602088C00506D56E
:1076A000E968032000048143A0690143E960207870
:1076B000000606D5E868032189048843E169084388
:1076C000E8600020F8BD00004010024000100240B9
:1076D0000070004088130000F8B504460D46002CE9
:1076E0001BD076480068C007C00FA8421CD2734F59
:1076F00038684008400028433860FFF7EDFC064634
:107700003868C007C00FA8420ED0FFF7E5FC811B08
:107710006B48814203D90320F8BD0120F8BD3868C9
:10772000C007C00FA842F0D12078664F800705D56A
:10773000F868F0218843A1680843F8602078C00702
:1077400072D06068022808D003280BD001280ED020
:107750003968890510D40120F8BD396889030BD434
:107760000120F8BD3968890106D40120F8BD3968C7
:10777000490701D40120F8BDF9688908890001434F
:10778000F960FFF7A9FC0646606802280FD00328BD
:1077900020D0012831D0F8680007800F44D0FFF7CF
:1077A0009BFC811B464881423AD90320F8BDF8680A
:1077B0000007800F022837D0FFF78EFC811B40485E
:1077C000814201D90320F8BDF8680007800F022824
:1077D000F2D129E0F8680007800F032824D0FFF7D2
:1077E0007BFC811B3648814201D90320F8BDF86833
:1077F0000007800F0328F2D116E0F8680007800F19
:10780000012811D0FFF768FC811B2D48814201D966
:107810000320F8BDF8680007800F0128F2D103E0CB
:10782000F8680007800FBAD124480168C907C90F5A
:10783000A9421CD90068214940084000284308603B
:10784000FFF74AFC06461D480068C007C00FA84263
:107850000DD0FFF741FC811B1948814201D903205B
:10786000F8BD16480068C007C00FA842F1D12078C3
:10787000400706D5F868072109028843E1680843F4
:10788000F8602078000707D5F8680721C902884307
:107890002169C9000843F86000F042F8F9680A4A13
:1078A0000906090F515CC84008490860084800688B
:1078B000FFF742FC0028D3D1F8BD000000200240B1
:1078C00088130000001002406CD20008080100205C
:1078D00000010020014800687047000008010020F6
:1078E00000B5FFF7F7FF0449C968044A4905490F85
:1078F000515CC84000BD00000010024085D2000865
:1079000000B5FFF7E7FF0449C968044A8904490F35
:10791000515CC84000BD00000010024085D2000844
:1079200070B5214EF2680C21104608401F498B00AB
:1079300004280CD04D00082810D00C2810D07068F6
:107940000004410F491C0120C003884070BD30680D
:10795000C00601D5084670BD184670BD284670BDEA
:107960009002134C000F205C1202940F641CF2680A
:10797000D20307D5294604F092FD22460023FDF7E5
:10798000CDFB70BD3268D20606D504F088FD2246D4
:107990000023FDF7C3FB70BD194604F080FD2246AD
:1079A0000023FDF7BBFB70BD0010024000093D0045
:1079B0007CD20008F0B583B00446002C0FD0F84EFE
:1079C000F5680C200540F768012000040740207886
:1079D000C0075BD0082D09D00C2D03D00FE001208B
:1079E00003B0F0BD01200004874208D13068800355
:1079F0004CD56068002849D1012003B0F0BD0120BA
:107A000061680004814203D131680143316015E0AF
:107A1000052301221B049204994206D131681143C7
:107A2000316031680143316008E031688143316081
:107A300031680140019130689043306060680028EF
:107A400012D0FFF749FB0290306880031ED4FFF785
:107A500043FB0299401A642802D9032003B0F0BD09
:107A600030688003F3D511E0FFF736FB02903068F1
:107A700080030BD5FFF730FB0299401A642802D926
:107A8000032003B0F0BD30688003F3D42078800772
:107A900068D5E068810604D5326820210A43326047
:107AA00088430923042D17D00C2D01D1002F13D0AA
:107AB000002842D03168994301433160FFF70CFB45
:107AC0000746306840072FD4FFF706FBC01B02288B
:107AD00027D9032003B0F0BD3168490701D500283C
:107AE0001CD071681F2212029143226912021143B5
:107AF00071603168994301433160FFF711FFF1680C
:107B000009060A0FA749895CC840A7490860A74829
:107B10000068FFF711FB0028DCD123E0012003B04F
:107B2000F0BD30684007CFD570681F210902884337
:107B3000216909020843706014E030684008400081
:107B40003060FFF7C9FA0746306840070AD5FFF7EB
:107B5000C3FAC01B022802D9032003B0F0BD30686D
:107B60004007F4D42078C0066BD5002D15D0A0694D
:107B7000002850D03068FF21013108433060FFF702
:107B8000ABFA07463068800536D4FFF7A5FAC01B6C
:107B900002282ED9032003B0F0BD3068800502D53D
:107BA000A069002822D07068072149038843216A10
:107BB000084370607068217F0002000A09060843CC
:107BC0007060206A410B491C0120C0038840F168A5
:107BD00009060A0F7349895CC840734908607348F5
:107BE0000068FFF7A9FA0028D5D12AE0012003B0E8
:107BF000F0BD30688005C8D5706807214903884307
:107C0000216A084370607068217F0002000A09063B
:107C10000843706015E03168FF2001308143316016
:107C2000FFF75AFA0746306880050AD5FFF754FA7D
:107C3000C01B022802D9032003B0F0BD30688005C4
:107C4000F4D420785A4F00072FD56069002816D049
:107C50003869012108433861FFF73EFA029038691C
:107C6000800722D4FFF738FA0299401A022802D975
:107C7000032003B0F0BD38698007F3D515E03869FB
:107C8000400840003861FFF727FA02903869800702
:107C90000BD5FFF721FA0299401A022802D90320D6
:107CA00003B0F0BD38698007F3D42078400775D55C
:107CB00000200190B06BC00006D4B06B0121090711
:107CC0000843B063012001903A480168C90519D4FE
:107CD0000068FF210131084336490860FFF7FCF9CD
:107CE000029034480068C0050CD4FFF7F5F90299FA
:107CF000401A642802D9032003B0F0BD2D48006863
:107D0000C005F2D5FF20A2680130824203D1396953
:107D1000014339611BE001218902002A0AD00523B1
:107D20001B029A420DD13A690A433A61396901430B
:107D300039610CE03A6982433A61386988433861B5
:107D400005E03A6982433A61386988433861A0683E
:107D5000002813D0FFF7C0F902903869800530D4AD
:107D6000FFF7BAF90299411A1348814202D9032058
:107D700003B0F0BD38698005F2D522E0FFF7ACF919
:107D80000290386980051CD5FFF7A6F90299411ABF
:107D90000948814212D9032003B0F0BD19E0000068
:107DA000001002406CD200080801002000010020F1
:107DB00040100240007000408813000038698005C0
:107DC000E2D40198012804D1B06B0121090788434E
:107DD000B063606A002864D00C2D49D001252D06BF
:107DE00002280FD03068A8433060FFF775F90446C9
:107DF0003068800155D5FFF76FF9001B022833D991
:107E00000320C9E73068A8433060FFF765F90746EB
:107E10003068800109D5FFF75FF9C01B022801D93E
:107E20000320B9E730688001F5D4E16AA06AF268FE
:107E30000843216BFD231B049A4311430843F06060
:107E4000306828433060FFF747F904463068800106
:107E500027D4FFF741F9001B022801D903209BE733
:107E600030688001F5D51CE030688001C3D418E08B
:107E7000012814D0F06801210904A26A014091424E
:107E80000BD10F218904E26A0140914205D10321FF
:107E900089050840216B884203D001207CE701203E
:107EA0007AE7002078E700000248016902221143C6
:107EB0000161704700E000E070B50446002C10D06E
:107EC00002202546403568742068016840229143AD
:107ED0000160204600F064F8002060656874287432
:107EE00070BD012070BDF8B50446002C0ED0FF27F0
:107EF000606A0537002600280AD026616661A662FE
:107F000025464035687C002807D00AE00120F8BDEE
:107F10006068B842F3D0E661F1E72E74204600F0C5
:107F200053F8022169742068026840239A43026072
:107F30002123A26860689B021A4038401043E3681E
:107F40008A021340184323690B40217D1843C90757
:107F5000C90F0843A169931019400843E169382308
:107F600019400843216A802319400843A16A9300FD
:107F70001940084321680860A0690421000C0840EA
:107F8000616A102319400843216848602068C1696C
:107F90009143C1616665012068740020F8BD00004E
:107FA00010B500680649884209D10648416B821421
:107FB000914341630520E0210007FEF73BFF10BD20
:107FC000003001400010024010B586B00446142174
:107FD0006846FDF7ECF810492068884219D10F482F
:107FE000416B821411434163C16A01221143C16292
:107FF000C06A002110400590E0200090022001900E
:108000000320039002910491052069460007FEF7C2
:108010009BFF06B010BD0000003001400010024080
:1080200010B40B49401E884202D910BC0120704791
:108030000849486108480723C2691202120A4C0421
:108040002243C261002088610B6110BC70470000B0
:10805000FFFFFF0000E000E004ED00E002480169DE
:10806000022291430161704700E000E0F0B4024653
:108070002032137E012B22D001261676022353765E
:1080800003685D689C687027BD430F682F435F607D
:108090000068B307984208D00A4B984205D00A4BB3
:1080A000984202D0094B984204D180239C434968EE
:1080B00021438160567600201076F0BC7047F0BCFA
:1080C00002207047000400400008014000140140F5
:1080D00010B5022104462034617601680A6A094B12
:1080E0001A4203D10A68520852000A6000F02CF8C4
:1080F0000020A077A076E076207760776076207603
:1081000010BD00001111000070B50546002D05D00E
:108110002C462034607E002802D006E0012070BD8D
:1081200000202076284600F01DF802206076291DE8
:10813000286803F077F80120A077A076E076207712
:1081400060776076002070BD00680449884204D1E1
:108150000348416B0422914341637047000801408A
:108160000010024000680449884204D10348416B72
:10817000042211434163704700080140001002408F
:10818000014620314A7E012A01D001207047022297
:108190004A760168CB6801221343CB6000689107DF
:1081A000884208D00B49884205D00B49884202D04A
:1081B0000A49884208D181684907490F062906D033
:1081C00001681143016002E0016811430160002071
:1081D0007047000000040040000801400014014006
:1081E0000168CA6852085200CA6001680A6A064BF0
:1081F0001A4203D10A68520852000A600121203055
:10820000417600207047000011110000F8B50446C7
:10821000002625462035287E012817D00120287603
:1082200002206876206882687727BA43FF231B0202
:108230009A4382600868502838D00EDC202853D03A
:1082400006DC002850D010281ED14DE00220F8BDD9
:10825000302849D0402817D13CE0602830D0702821
:1082600019D001221203801A0FD090420CD1CB6892
:108270004A688968206803F017F82068816801223D
:1082800092031143816000E00126012068760020FE
:1082900028763046F8BDCB684A688968206803F0C4
:1082A00003F82068816839438160EEE7CA6849684D
:1082B000206803F07EF85021206803F001F8E4E71D
:1082C000CA684968206803F086F86021206802F0D7
:1082D000F7FFDAE7CA684968206803F06AF84021C6
:1082E000206802F0EDFFD0E722680146104602F058
:1082F000E7FFCAE710B586B0044614216846FCF7CC
:1083000056FF0D492068884213D10C48C26A0221E9
:108310000A43C262C06A01910840059008030090B8
:108320000020029003900620049069460448FEF75E
:108330000BFE06B010BD0000000801400010024016
:1083400000040050F8B504460D46002726462036A6
:10835000307E01280ED001203076002A0CD0042A6D
:108360001ED0082A33D00C2A45D0012700203076B1
:108370003846F8BD0220F8BD2946206802F0A8FF63
:108380002068816908221143816120688169042283
:108390009143816120688169EA6811438161E5E761
:1083A0002946206802F0ADFF206882690121C902D8
:1083B0000A438261206881690122920291438161AE
:1083C00020688169EA68120211438161CEE729467B
:1083D000206802F0B3FF2068C16908221143C1611F
:1083E0002068C16904229143C1612068C169EA68BB
:1083F0001143C161BAE72946206802F0BBFF20683B
:10840000C1690122D2021143C1612068C269012100
:1084100089028A43C2612068C169EA681202114375
:10842000C161A3E770B50546002D05D02C46203468
:10843000607E002802D006E0012070BD002020767A
:10844000284600F00FF802206076291D286802F007
:10845000E9FE0120A077A076E0762077607760764D
:10846000002070BD7047000070B505462C462034D2
:10847000002908D0042908D0082908D0627F012AE1
:1084800007D0012070BDA27EF9E7E27EF7E7227FE8
:10849000F5E70220002920D0042920D0082920D087
:1084A00060770122286802F0F1FE0121286889071F
:1084B0000122884208D00E49884205D00D498842E1
:1084C00002D00D4988420ED181684907490F06291B
:1084D0000CD001681143016008E0A076E1E7E07686
:1084E000DFE72077DDE7016811430160002070BD00
:1084F00000040040000801400014014070B504462B
:108500000D4600222946206802F0C0FE2068016A5C
:108510000B4A114203D1016849084900016001205A
:108520002034002D06D0042D06D0082D06D060770B
:10853000002070BDA076FBE7E076F9E72077F7E74B
:10854000111100007047704770B50446002C1BD015
:108550002420E0672068016849084900016020681C
:10856000002505602068456020688560204600F091
:108570009BF9204680304560E567056025666566A5
:1085800060342576002070BD012070BD10B503F069
:10859000D5FD10BDF8B504462268D069116893680E
:1085A000A24D06462E40002E09D1850607D58D0620
:1085B00005D5A16E002901D020468847F8BD254683
:1085C0008035002E7FD09A4FDE07F60F0F403743DD
:1085D00079D0C70706D0CF0504D5012717626A688E
:1085E0003A436A60820708D5DA0706D02768022274
:1085F0003A626A6804273A436A60420708D5DA0794
:1086000006D0236804221A626A6802231A436A6049
:10861000020709D520220A40324305D023680822E8
:108620001A626B6813436B60020509D54A0107D5CE
:1086300001222368D2021A626A6820231A436A6000
:108640006A68002ABAD0800606D5880604D5A16ECD
:10865000002901D020468847686821688968490652
:1086600002D42821084228D0204603F05FF8206871
:10867000816849061DD5EFF31081012282F310882D
:10868000836840229343836081F31088606F0028E1
:108690000BD068498163606FFEF7BFFA00288DD068
:1086A000606F816B8847F8BD0DE02046FFF76EFFD5
:1086B000F8BD2046FFF76AFFF8BD2046FFF766FFCA
:1086C00000206860F8BD266E012E7DD1C6067BD5E0
:1086D000CE0679D5102313622068816826464906A4
:1086E000403600294CDA626F1168496889B2002966
:1086F000E8D0378B8F42E5D9718311680968890604
:1087000034D4EFF31081012282F3108802681F0134
:10871000BA43026081F31088EFF31081012080F3E7
:1087200010882068826852085200826081F31088A5
:10873000EFF31081012080F31088206882684027C1
:10874000BA43826081F310882020286000202066D0
:10875000EFF31081012080F31088206802689A43AB
:10876000026081F31088606FFEF733FA02206066C2
:10877000308B718B401A81B22046FFF7E3FEF8BDC3
:10878000318B728B891A89B2728B002AF7D000293B
:10879000F5D0EFF31082012686F310880668FF27D4
:1087A0002137BE43066082F31088EFF31082012068
:1087B00080F310882068866876087600866082F3E9
:1087C00010882020286000E013E000202066A066CA
:1087D000EFF31082012080F31088206805689D4324
:1087E000056082F31088022060662046FFF7AAFE2B
:1087F000F8BDC50208D55B0206D501200005106250
:108800002046FFF7A0FEF8BD020607D50A0605D5EB
:10881000E16E0029F7D020468847F8BD4006FCD518
:108820004806FAD5204602F0B1FFF8BD0F08000057
:1088300020010004BDB5000810B50446002C03D08B
:10884000E06F002802D007E0012010BD0021782051
:108850000155204600F064F82420E0672068016894
:10886000490849000160204603F092F8012819D018
:10887000606A002802D0204602F0D2FD20684168DC
:108880000922D20291434160206881682A229143E3
:10889000816020680168012211430160204602F0D6
:1088A00025FE10BD012010BD10B5026817481849FB
:1088B00082420BD1886B012292049043886303218A
:1088C00089021448FEF7B6FA1D200EE0124B05206F
:1088D00000079A420CD14A6B01239B039A434A63D7
:1088E00003214902FEF7A6FA1B20FEF7B1FD10BDD9
:1088F0000A4B9A42FBD18A6B01235B049A438A6339
:108900000C21FEF797FA1C20EFE70000004800401A
:1089100000100240000400500038014000440040B4
:10892000F0B587B0044614216846FCF740FC314A94
:10893000266800253048022103230424964218D1DA
:10894000826B4E0432438263C26A0A43C262C06AC7
:108950006A4608400590980223C218C26946274813
:10896000FEF7F2FA002211461D20FEF78DFD1D20B4
:108970001CE0234F0122BE421CD1456B96033543B8
:108980004563C56A1543C562C06A6D4610400590CF
:10899000032040021FC5052069460007FEF7D4FAF0
:1089A000002211461B20FEF76FFD1B20FEF760FD25
:1089B00007B0F0BD134FBE42FAD1866B01277F048A
:1089C0003E438663C66A1643C662C06A6E46C007E7
:1089D000C00F05900C2023C6052018C66946000765
:1089E000FEF7B2FA002211461C20FEF74DFD1C20B6
:1089F000DCE7000000480040001002400004005086
:108A0000003801400044004070B580231B58202BE3
:108A100001D0022070BD00290AD0002A08D001240C
:108A200083682403A34209D10369002B02D005E027
:108A3000012070BDCB0701D0012070BD002303666B
:108A40000A4C0368A3420ED05C6824020BD5EFF3F6
:108A50001084012585F310881D680126B60635436C
:108A60001D6084F3108803F0CDF870BD004800400D
:108A700070B580231B58202B01D0022070BD002927
:108A80000AD0002A08D0012483682403A34209D114
:108A90000369002B02D005E0012070BDCB0701D097
:108AA000012070BD002303660A4C0368A3420ED068
:108AB0005C6824020BD5EFF31084012585F3108840
:108AC0001D680126B60635431D6084F3108803F047
:108AD000F1F870BD0048004010B503F051FB10BD27
:108AE0007047FFB583B004460F461546E06F202857
:108AF00002D0022007B0F0BD002F0AD0002D08D010
:108B00000120A168000381420BD12069002803D015
:108B100007E0012007B0F0BDF80702D0012007B040
:108B2000F0BD0021842001512120E067FEF7D4FA36
:108B3000029026464036358275820120A1680003E6
:108B4000814202D12069002813D03D460027708A57
:108B500000281CD006980090002280212046029B0D
:108B600003F078F9002806D02020E067032007B042
:108B7000F0BD0025EBE7002D18D021682878886229
:108B80006D1C708A401E7082708A0028E2D106989F
:108B90000090002240212046029B03F05BF9002850
:108BA0000BD02020E067032007B0F0BD3888216893
:108BB000C005C00D8862BF1CE3E72020E0670020ED
:108BC00007B0F0BD70B50446E06F202801D0022048
:108BD00070BD00290AD0002A08D00123A0681B0319
:108BE000984209D12069002802D005E0012070BD1B
:108BF000C80701D0012070BDE164204640300282E8
:108C0000428200214030054641602120E067206F0C
:108C100000281AD0154BC362236F15481863236FC1
:108C200014485863206F8163206813462830266FEC
:108C300002463046E16CFEF716F8002805D01020F9
:108C400068602020E067012070BD21684020086234
:108C5000EFF31081012080F3108820688268802360
:108C60001A43826081F31088002070BDD7B60008D7
:108C700023B70008D1B5000830B4C36F202B02D051
:108C800030BC0220704700290AD0002A08D00124F5
:108C900083682403A3420BD10569002D03D007E0AC
:108CA00030BC01207047CD0702D030BC0120704796
:108CB000C164014640310A824A820021C166842291
:108CC00011502121C167A34202D10169002910D0AE
:108CD0000949C166EFF31081012282F31088006810
:108CE000026880231A43026081F3108830BC0020A0
:108CF00070470249C166EDE7F7BD000895BD000861
:108D000010B503F0D5FA10BD7047000000200149EE
:108D100008707047B00300200120014908707047B7
:108D2000B003002070B504460D46204600F02CF834
:108D3000012801D1801E70BD2268501CE168FCF73B
:108D4000D7F92160236921685943A368C8182946C7
:108D50002269FCF713FA0020EDE710B58160C260CC
:108D60000361012444600024046010BD10B5044672
:108D70002268501CE168FCF7BBF96068814201D1B0
:108D8000012010BD0020FCE710B504462268901CAD
:108D9000E168FCF7ADF96068814201D1012010BDA6
:108DA0000020FCE770B504460D462046FFF7DEFFC5
:108DB000012801D1801E70BD236960685843A368F3
:108DC000C11828462269FCF7D9F96268501CE1688D
:108DD000FCF78EF961600020EDE770B504460D46A2
:108DE000002C01D1401E70BD00BF2068A842FCD3FA
:108DF0002068401B206062685019E168FCF778F930
:108E000061600020EFE770B504460D46002C01D1EB
:108E1000401E70BD20684019206000BFE1682068D6
:108E20008842FBD8A2685019E168FCF761F9A1609B
:108E30000020EEE7FFB581B004460D461646002738
:108E4000002E06D00498002803D0E16820688842EC
:108E500003D30020C04305B0F0BD2168E068401A8C
:108E6000A84202D20020C043F5E7A0684019E1689B
:108E700088420BD9A168E068471A2168E068401A67
:108E8000E919884202D20020C043E4E7A268D01961
:108E9000E168FCF72DF93160791904980160002030
:108EA000D9E701464868704701468868704702461E
:108EB000002A01D1401E7047002050609060106071
:108EC000D16000BFF7E70146002901D101207047BA
:108ED0000868002801D10120F9E70020F7E70146E2
:108EE000002901D1012070470A68C868904201D169
:108EF0000120F8E70020F6E70FB400B50D48FFB0F9
:108F0000007882B0012805D000207FB002B008BCF4
:108F100004B01847012183AB49026846829A03F0E6
:108F200091FA6846FCF762F902466946002003F0B0
:108F300053F9EAE78800002010B5064A1278012AA2
:108F400001D0002010BD0A460146002003F044F97C
:108F500010BD00008800002003490968016002215B
:108F600081710149086070472001002000BFEFF3C4
:108F70000580002800D0704707480068002804D109
:108F8000012080F3108800BF00BF03480068401C28
:108F90000149086000BFEEE70C01002070B50446EF
:108FA0000D4600F04FF800280FD000F04BF80B21D1
:108FB000C90140180069002807D000F043F80B22CF
:108FC000D2018018016902A08847002070BD00000E
:108FD0001B5B481B5B4A000070B502460C46002133
:108FE0000023002A01D0002C02D10020C04370BD14
:108FF0000021002316E0C8000D4D2858002810D18C
:10900000D8001058CD000A4E7051D8008018406822
:10901000CD00AD19686007480068401C054D286008
:109020005B1C491C502901D2A342E4D30020DEE797
:109030002C01002028010020014800687047000032
:10904000280100200148006870470000240100202A
:10905000F8B506460F46002536E0002418E0FFF775
:10906000F1FF002813D0FFF7EDFF0B21C9014018D5
:10907000006900280BD0FFF7E5FF0B23DB01C018C8
:1090800002692819C000134B195813A09047641C9B
:10909000052C04DAFFF7D0FF29198842DFD8FFF743
:1090A000D1FF00280FD0FFF7CDFF0B21C9014018D9
:1090B0000069002807D0FFF7C5FF0B22D2018018F6
:1090C000016907A088476D1DFFF7B6FFA842C4D805
:1090D0000020F8BD2C010020252D31367300000042
:1090E0000D0A00000146202902D30020C04370472A
:1090F000012218204843044B1A50002218204843EC
:10910000C01882600020F2E7A029002070B5054653
:109110000024002D01D1401E70BD00240CE0182059
:1091200060430C490858002805D1012118206043EC
:10913000084A115002E0641C202CF0D300BF202C00
:1091400005D105A0FFF7D8FE0020C043E4E72C605E
:109150000020E1E7A029002074696D657220494470
:109160002069732066756C6C0D0A000010B5002430
:1091700000BF41E0182060432149085802283AD135
:1091800018206043401880681E490968091A182091
:1091900060431B4A8018C06881422CD91820604364
:1091A000114640184069002820D01820604340181C
:1091B0000079002804D101211820604311500AE0F1
:1091C0000221182060430E4A11500E4801681820F1
:1091D00060438018816018226243094BD2181069DD
:1091E00018226243D2185169884704E001211820EF
:1091F0006043034A1150641C202CBBD310BD0000F7
:10920000A029002010010020F0B50446059D202C67
:1092100002D30020C043F0BD0226182060430E4F49
:109220003E50182060433E46801901710B48066885
:1092300018206043C0198660182060433E4680199C
:10924000C260182060438019436118206043801970
:1092500005610020DFE70000A029002010010020A8
:1092600007480068401C06490860064802684068D4
:109270000021521C484103490A60486070470000C1
:10928000100100201801002000BFEFF30580002826
:1092900000D0704709480068002804D007480068DB
:1092A000401E0649086005480068002804D100BF38
:1092B00080F3108800BF00BF00BFEAE70C01002068
:1092C00070B504460D4629462046FBF770FF70BD79
:1092D0000146302904DB392902DC084630380EE02B
:1092E000412904DB462902DC0846373807E06129BA
:1092F00004DB662902DC0846573800E00020C0B2D3
:10930000704710B502460B46002406E01078FFF7C0
:10931000DFFF21014418521C5B1E002BF6D12046B2
:1093200010BD0FB4F0B585B00446002004900022B3
:109330002020039000200290002C02D00C980028DE
:1093400005D1002005B0F0BC08BC04B018470DA83A
:109350000490CFE0002908D10C980078252803D18B
:109360000C984078652800D0C9E00C980078252832
:109370006ED10C98401C0C900C98007803900C98BF
:10938000401C0C900398652877D004DC2A2807D06D
:10939000642873D113E0702872D07828F9D13EE0A8
:1093A00008E020780C9B1B78984202D0641C491E70
:1093B00000E001E00029F4D100BF521C88E0002643
:1093C00001960096002300252020049E20CE0496BE
:1093D00018E02078009E002E05D12D2803D101260B
:1093E000019600960CE0302809DB392807DC0126BD
:1093F00000960A265E430746303FF31900E003E07B
:10940000641C491E0029E4D100BF019E012E01D138
:10941000DE43731C002D00D02B60521C58E000234B
:109420000025049E20CE04961FE02078302806DB1D
:10943000392804DC1E010746303FF31913E0612888
:1094400007DB662805DC1F010646573EBB190AE00C
:1094500043E0412806DB462804DC1F010646373E70
:10946000BB1900E003E0641C491E0029DDD100BFE8
:10947000002D00D02B60521C2AE01BE024E0FFE707
:10948000049E01CE049600250023254609E0267897
:109490000C9F3F78BE4201D05B1C00E003E0641CDF
:1094A000491E0029F3D100BF002801D005604360A8
:1094B000521C0DE0049B01CB0493002800D00460F3
:1094C000521C0123029303E001200290002200BFFE
:1094D00000BF029801280DD111E020780C9B1B7869
:1094E000984205D1641C0C98401C0C90491E01E068
:1094F000002204E00C980078002800D02AE700BF82
:109500000020049010461DE70FB4F8B506460C463F
:10951000002509A8009021463046009B089A02F0D9
:1095200091FF054600200090A54200D3651E284605
:10953000F8BC08BC04B01847FEB504460F461546F3
:109540000026002001900090002C01D0002D01D1B8
:109550000020FEBD2846FBF749FE00900098874298
:1095600001D20020F5E70098381A0190002609E0A2
:10957000A0192946009AFBF740FE002801D1A01946
:10958000E7E7761C01988642F2D30020E1E770B548
:1095900004460D46002C01D0002D02D10020C0430E
:1095A00070BD012120461030FFF717FC2046203007
:1095B000A968FFF712FC0020F2E770B504460D46DB
:1095C000002C01D0002D02D10020C04370BD01212C
:1095D00020461030FFF717FC20462030A968FFF71F
:1095E00012FC0020F2E710B50446002C00D110BD9B
:1095F00020461030FFF767FC012801D10020F6E774
:1096000020462030FFF75FFC012801D10020EEE763
:1096100020461030FFF745FC0C21484321684018D4
:10962000E5E77CB504460E46002500200190009039
:10963000002C00D17CBD20461030FFF750FC0028E4
:1096400001D00020F6E76B4601AA314620462030C3
:10965000FFF7F0FB002801D00020EBE72046103098
:10966000FFF722FC0C21484321684518A0680199A6
:10967000401828606E600098A8602846DAE7FFB5B9
:1096800081B004460E461D4600270C20684303990E
:10969000884202D3781E05B0F0BD0C202F46474308
:1096A0002660676060688019A0600398C11BE16054
:1096B000294620461030FFF7FAFB20462030E168AB
:1096C000FFF7F5FB0020E6E7FEE7000010B50E4CC3
:1096D000002208212046FDF7F8FC00221021204638
:1096E000FDF7F3FC0A2003F08BFB01220821204642
:1096F000FDF7EBFC0A2003F083FB00220821204643
:10970000FDF7E3FC10BD00000004005010B50E4C46
:10971000002208212046FDF7D8FC01221021204616
:10972000FDF7D3FC0A2003F06BFB01220821204641
:10973000FDF7CBFC0A2003F063FB00220821204642
:10974000FDF7C3FC10BD000000040050F8B5002474
:10975000144E07462546002208213046FDF7B5FC89
:109760000A2003F04DFB012208213046FDF7ADFC35
:109770006006040E10213046FDF7A0FC002801D041
:10978000641CE4B2052003F03BFB6D1CEDB2082D18
:10979000E1D3002F03D0FFF799FF2046F8BDFFF774
:1097A000B5FFFAE70004005070B5154E05460022DB
:1097B00008213046FDF789FC0024E80901D0012288
:1097C00000E0002210213046FDF77FFC6806050E00
:1097D0000A2003F015FB012208213046FDF775FC35
:1097E0000A2003F00DFB002208213046FDF76DFC36
:1097F0000A2003F005FB641CE4B2082CDDD370BD25
:109800000004005010B50C4C012210212046FDF739
:109810005CFC012208212046FDF757FC00221021A4
:109820002046FDF752FC0A2003F0EAFA0022082144
:109830002046FDF74AFC10BD0004005010B50E4C48
:10984000002208212046FDF740FC0022102120467E
:10985000FDF73BFC0A2003F0D3FA01220821204641
:10986000FDF733FC012210212046FDF72EFC0A20D3
:1098700003F0C6FA10BD00000004005070B5144D8E
:109880000024012210212846FDF71FFC062003F0CA
:10989000B7FA012208212846FDF717FC062003F03D
:1098A000AFFA07E0641CE4B2FA2C03D9FFF7C6FF55
:1098B000012070BD10212846FDF700FC0028F1D1E1
:1098C000002208212846FDF700FC002070BD0000A2
:1098D0000004005010B5FCF779FC10BD70B500F025
:1098E0002FF80025104C012818D16078002815D1D8
:1098F000012060700D480E49056020780D4B0E4A1E
:109900000E4E5A2802D3FF20000401E0FF2000027F
:1099100008601B681268316801F044F900F010F823
:10992000002800D1657070BD380000202C00002098
:1099300024000020180000201C000020200000202F
:1099400010B5044881880068FDF7B8FB012800D0F5
:10995000002010BD5000002010B53721202000F05D
:1099600070F80321212000F06CF84021222000F043
:1099700068F80821232000F064F8AA21302000F0C4
:1099800060F80A4802210187322000F05AF80121CC
:10999000332000F056F85F21202000F052F80448F0
:1099A00000F008F80A2003F02BFA10BD740600201E
:1099B000DB00002010B501460F2000F021F8002840
:1099C00000D0012010BD10B50446FFF71BFF322068
:1099D000FFF7EAFEFFF752FFE0B2FFF7E5FEFFF701
:1099E0004DFFFFF70FFF3320FFF7DEFEFFF746FFC7
:1099F0000020FFF7ABFE0446FFF720FF204610BD16
:109A000010B50C46FFF7DFFF2070012010BD70B5C8
:109A10000D460446FFF7F6FE3220FFF7C5FEFFF7BE
:109A20002DFFE0B2FFF7C0FEFFF728FF2846FFF743
:109A3000BBFEFFF723FFFFF701FF0A2003F0E0F969
:109A400070BD10B5FFF7E3FF012010BD10B502484F
:109A5000FDF7CCFB10BD000014040020F0B583B06E
:109A600004460026EFF310800090012080F3108858
:109A7000344B2068C21804D13349CE6803218904CD
:109A80000E4081680291C168019141698569002A8F
:109A900007D12E48826AC7043A438262826ABA4377
:109AA0008262084628433CD026482268C24205D13B
:109AB0002548C368032292049343C3602746203796
:109AC000002910D02068026901231A43026120682E
:109AD00041610821204600F03BF8032800D1B8730B
:109AE000216808204860002D10D0206801690122FB
:109AF00011430161206885611021204600F028F89B
:109B0000032800D1B8732168102048600D482168EF
:109B1000C14206D10C48C1680322920491433143EB
:109B2000C160206801694908490001612168029803
:109B3000886021680198C860009880F3108803B09D
:109B4000F0BD00000084FFBF401002400010024042
:109B500070B506460D4600240B480A490068FBF71D
:109B6000C7FA7D21C90048433268401E002800D151
:109B7000032413682946994301D00028F5D12046D3
:109B800070BD0000204E00000801002010B5024802
:109B9000FEF700FD10BD00004404002010B50320B6
:109BA00000F002F810BD000070B5164D00262C46DE
:109BB000103C002811D021468978032814D00128B0
:109BC0000AD1491CC8B2A0700C2817D204280FD0A3
:109BD0008000285800F0B0F970BD00F049FA052067
:109BE000FDF77AF8A67001E00029F5D12868F1E7C1
:109BF00005492869096800F09FF970BD00F02EFA48
:109C000070BD0000A40000205C00002000B587B0FB
:109C1000012069464870022008700E4901914102F6
:109C200002910D490391802104910590694601201C
:109C300002F0BAF90948FFF769FA00F019FA00F0E2
:109C40006BF96420FDF748F80020FFF7ADFF002016
:109C500007B000BD2C2300202C2700209C000020F2
:109C6000034880780C2801D00020704701207047FD
:109C700094000020032802D30020C0437047C30093
:109C80000248C15018188280002070471423002019
:109C9000FEB5002568460571058105805D4F5E4C67
:109CA0005E4EA0E06846007900F0EAF86846017967
:109CB00030782154401C307020785528F1D16078DC
:109CC000AA28EED1607A5528EBD1A07AAA28E8D14B
:109CD0006068029052496846008909688842E0D16C
:109CE000A079012814D1E07901287CD1207A0028BC
:109CF00079D14C4805604C4805704C4805704CA023
:109D0000FFF7FAF8FF2101314348FBF750FA3570AD
:109D1000A079022806D0032818D0052826D00428C8
:109D200061D141E03C496846CA790270097A4170C4
:109D300000883C2802D83C20694608806846048890
:109D4000BC8403F02DFA21463DA026E03249684646
:109D5000CA790270097A417000880A2802D80A205C
:109D600069460880684604887C8712E02A4968466C
:109D7000CA790270097A417001887D20C000081AF2
:109D80003649884202D336486946088068460488C6
:109D9000FC8003F005FA214632A0FFF7ADF86420FD
:109DA00003F027F802F0A2FB1B486946C2790A704B
:109DB000007A487008880A2801D80A2002E064283E
:109DC00001D964200880088830710120707116481C
:109DD000FF210570154801310570124805600E48D5
:109DE000FBF7E5F9357001A9012002F09DF8002884
:109DF00000D157E7FFF734FF012809D1F078002898
:109E000006D0FF2101310448FBF7D1F9F570357018
:109E1000FEBD0000740600201422002094000020E3
:109E20005C00002058000020740000207500002015
:109E3000CAD5B5BD475053B5C44F4B0D0A000000FD
:109E4000CAD5B5BDD0DEB8C4475053BFAAB9D8CA29
:109E5000B1BCE43A25640D0A00000000292300008B
:109E600010270000CAD5B5BDD0DEB8C4BEB2D6B981
:109E7000D0DDC3DFCAB1BCE43A25640D0A0000009E
:109E800070B51E491E4B4A78012A05D1CA687F2A3F
:109E900002D29854521CCA6000220A2802D00D280F
:109EA00004D029E00120CA60487025E04A70CC68DF
:109EB000002C21D018192038C277114D8868FFF77F
:109EC00011F910A221462846FFF736FB002805D0DD
:109ED00029460DA0FFF710F801200BE00CA2214647
:109EE0002846FFF729FB002806D0294606A0FFF7E1
:109EF00003F80220FFF758FE002070BD94000020F8
:109F0000AC2700206F6B00005B525D2025730A00B8
:109F10006572726F7200000010B5034801228188DB
:109F20000068FDF7D2F810BD1423002010B5002002
:109F3000FFF73AFE10BD00000FB430B591B015AB7D
:109F4000402101A8149A02F07DFA002501A8FBF730
:109F50004DF9024601A9012002F03EF904460A48E3
:109F60007D220095074B120100218068FFF74CF914
:109F700001A906A0FEF7C0FF204611B030BC08BC06
:109F800004B018479D9B0008940000205B535D209F
:109F900025730A0070B505460C480C4680780C28DD
:109FA00002D00020C04370BD00F062F80520FCF72D
:109FB00093FE22462946012002F00EF90520FCF707
:109FC0008BFE00F04BF8002070BD000094000020D4
:109FD000F8B5184E184D3068E968401A012828D99C
:109FE000164801781648FFF7D5FFFF2101311548C3
:109FF000FBF7DDF81448002404703068E860287925
:10A00000FF21401C2871114D12482960104E124F3B
:10A0100002683368386800F0C5FD6420FCF75CFE18
:10A020002C603C600B48336802682146204600F0F3
:10A03000B9FDF8BD28000020380000208E00002067
:10A04000EC110020142200209400002020000020A9
:10A05000180000201C0000202400002010B5034838
:10A06000002281898068FDF730F810BD142300209C
:10A0700010B50348012281898068FDF726F810BDDC
:10A08000142300201CB5002118480091164A0191A4
:10A090000260C1631205426081600722826301226F
:10A0A00002610246C16020321170FF235170C23339
:10A0B00043628162117301638161042241634261E1
:10A0C000C161FCF7ADFB002801D072B6FEE708487D
:10A0D00000908013019069460448FCF7F3FA0028C9
:10A0E00001D072B6FEE71CBD00240140B803002079
:10A0F00002000004F0B587B014216846FBF757F85A
:10A100004148C26A04210A43C262C26A0A400592F7
:10A11000C16A01252943C162C16A29400591C26A09
:10A1200002210A43C262C06A052708403F07059022
:10A13000002236493846FCF7C8FF0022344935482A
:10A14000FCF7C3FF012211033846FCF7BEFF0122D2
:10A1500040213048FCF7B9FF112636040024694637
:10A160003846019600950294FCF7EEFE2A480090CE
:10A1700002946946019503943846FCF7E5FE2448AD
:10A180000294183800906946019503942148FCF721
:10A19000DBFEA22000906946019602941D48FCF760
:10A1A000D3FE0920000300900194694602941948E7
:10A1B000FCF7CAFE18200090112001900294694615
:10A1C00003941448FCF7C0FE402000900320039045
:10A1D0000195029469460F48FCF7B6FE2802FCF789
:10A1E00081FF002211460520FDF74EF90520FDF7FD
:10A1F0003FF9002211460720FDF746F90720FDF739
:10A2000037F907B0F0BD00000010024010890000CF
:10A210001D410000000400501099000010B5FFF728
:10A2200031FF00F009F800F099F800F0B3F800F001
:10A230001FF800F043F810BD10B50C480A49016042
:10A24000E1214902416000218160C16001618161B9
:10A250000C22016242614162FEF7EEFA002801D051
:10A2600072B6FEE710BD0000004800404404002024
:10A2700010B5114C0F482060FF20053060600020B1
:10A28000A060E06020616061E0610121206249021C
:10A290006062A161A0620720E0622046FDF723FE14
:10A2A000002801D072B6FEE7206801684022114301
:10A2B000016010BD00300140DC05002010B58AB0FF
:10A2C0000024049405940694079408942248099461
:10A2D0000094019402941F49039401601F2184603B
:10A2E00041600461F9214461C160FDF70DFF002860
:10A2F00001D072B6FEE701200003049004A91648BD
:10A30000FDF784FF002801D072B6FEE71248FEF781
:10A3100089F8002801D072B6FEE7089408A90E4813
:10A320000994FDF7A3FE002801D072B6FEE7602075
:10A330000090019402940022694603940648FEF7B7
:10A3400001F8002801D072B6FEE70348FDF7D2FFFE
:10A350000AB010BD000801403406002010B50C48BA
:10A360000A490160E1214902416000218160C16028
:10A3700001618161C1610C22016242614162FEF7AB
:10A380005BFA002801D072B6FEE710BD003801402C
:10A39000CC04002010B50C480A4901604B21C901CA
:10A3A000416000218160C16001618161C1610C2255
:10A3B000016242614162FEF73FFA002801D072B6A5
:10A3C000FEE710BD0044004054050020FEE7704742
:10A3D00010B50448002281898068FCF776FEFCF7FE
:10A3E00023F910BD0422002010B504480122818900
:10A3F0008068FCF76AFEFCF71DF910BD04220020FE
:10A40000C3000248C15018188280704704220020FF
:10A41000F0B585B04848FCF7A3F94848FDF74CFD76
:10A420004748FDF755FE4748FEF78EF84648FEF7C9
:10A430008BF84648FEF788F800F0D0FB14216846F8
:10A44000FAF7B5FE0024102611270520029469466C
:10A450000007019700960394FCF776FDF5010520AF
:10A46000029469460007019700950394FCF76CFD80
:10A47000FDF7F4FD3648816B0204114381633548D2
:10A48000016804221143016001210846FDF726F806
:10A49000FDF70AFD00F064FEFFF7C0FE002001F0AA
:10A4A000FDFD012001F0FAFD022001F0F7FD00960C
:10A4B0000126052002946946000701960394FCF7E3
:10A4C00043FD0520012210210007FCF7FEFD0520B9
:10A4D000029469460007019600950394FCF734FD49
:10A4E0000520012229460007FCF7EFFD1A480078F5
:10A4F00000281CD1194C2068C10718D1184D2968B3
:10A50000884214D0174801781748142901D3FF2135
:10A5100001E0FF2109020160144900680B68144939
:10A520000A681449096800F03DFB2068286012A001
:10A53000FEF7E2FC05B0F0BDB8030020DC0500200A
:10A540003406002044040020CC04002054050020E0
:10A550000010024000700040300000202800002061
:10A5600034000020380000202400002018000020C3
:10A570001C0000202000002077616B752075700D95
:10A580000A000000F8B502F0C7FD754800F0CAFAED
:10A59000744CE0807248801C00F0C4FA208170483E
:10A5A000001D00F0BFFA608170486F494180818CC6
:10A5B000002902D1E12109018184418F6C4A0029DF
:10A5C00001D0914201D96B4941878BB2818C8B427A
:10A5D00002D2FF312D314187C3887D21C900591A2C
:10A5E000654B994200D3C280604D6048403529795F
:10A5F00061700091614AC18E1170614AC18F117002
:10A60000604A818F1170A97921705F4A817A117037
:10A610005E4986880E605E4A05211180C7883846EB
:10A62000FAF766FD5B49088001463046FAF760FD9F
:10A630008800081886B2584806807D20C000704304
:10A64000FBF768F8554A564BFAF7ECFFFBF784F82E
:10A65000544908805448068054480188C820FAF7B5
:10A6600047FD534900260880524901200880A780F1
:10A670000099002906D17D21C900A18040490870B8
:10A68000404806707D20A188C000FAF731FD474997
:10A690000022088048494948FCF77EFE002801D086
:10A6A00072B6FEE7A88C012805D0688C444C454F53
:10A6B000012838D03FE0FF20000203461A46114629
:10A6C00000F070FAFF24F5342046FCF705FBFF206C
:10A6D000000403461A46114600F064FA2046FCF7CF
:10A6E000FBFA00231A461946184600F05BFA20468A
:10A6F000FCF7F2FA34486946088072B68021334C80
:10A700002046FBF797FD002804D002226946204628
:10A71000FBF736FE62B6AE8402F042FD642002F022
:10A7200068FB01F0D5FE00F0CBF902F039FD6420A2
:10A7300002F05FFBFC60288C012806D12E8402F019
:10A740002FFD642002F055FBFC600848204A018878
:10A75000914202D1C088002800D1FC60F8BD000001
:10A76000004F0008000000200902000074060020CD
:10A77000102700003C0F000029230000F0000020FB
:10A780006E0000206F000020600000205C000020B0
:10A79000640000206600002062000020F853E3A55A
:10A7A0009B843E40680000206C0000206A0000206E
:10A7B0007200002070000020FF7F000014040020C1
:10A7C0000400FA0500ED00E0AAAA0000384A0008DB
:10A7D000AA55000000B5044940208862FF20F530EA
:10A7E00002F0FAFC00BD000000040050FF23024606
:10A7F0001B0200B519020D489A4202D100F0C0F8C0
:10A8000000BD8A4202D100F057F809E0FF2A04D0C7
:10A81000824205D100F002F900BD00F009F800BD48
:10A82000002AFCD100F07AF800BD0000FFFFFF0015
:10A8300000B500F02FF800F02DF800F02BF800F034
:10A8400029F800F027F800F025F800F023F800F0D0
:10A8500021F800F01FF800F01DF800F01BF800F0E0
:10A8600019F800F017F800F015F800F013F800F0F0
:10A8700011F800F0B7F800F0B5F800F0B3F800F008
:10A88000B1F800F0AFF800F0ADF800F0ABF800F070
:10A89000A9F800BD07484021816100BF00BF00BF8B
:10A8A00000BF00BF00BF816200BF00BF00BF00BF8C
:10A8B00000BF70470004005000B500F093F800F0AE
:10A8C00091F800F08FF800F08DF800F08BF800F0B0
:10A8D00089F800F087F800F085F8FFF7DBFFFFF755
:10A8E000D9FFFFF7D7FFFFF7D5FFFFF7D3FFFFF73C
:10A8F000D1FFFFF7CFFFFFF7CDFFFFF7CBFFFFF74C
:10A90000C9FFFFF7C7FFFFF7C5FFFFF7C3FFFFF75B
:10A91000C1FFFFF7BFFFFFF7BDFF00BD00B5FFF7A9
:10A92000B9FFFFF7B7FFFFF7B5FFFFF7B3FFFFF77B
:10A93000B1FFFFF7AFFFFFF7ADFFFFF7ABFFFFF78B
:10A94000A9FFFFF7A7FFFFF7A5FFFFF7A3FFFFF79B
:10A95000A1FFFFF79FFFFFF79DFFFFF79BFFFFF7AB
:10A9600099FFFFF797FFFFF795FFFFF793FFFFF7BB
:10A9700091FFFFF78FFFFFF78DFFFFF78BFF00BD04
:10A9800000B5FFF787FFFFF785FFFFF783FFFFF7AE
:10A9900081FFFFF77FFFFFF77DFFFFF77BFFFFF7EB
:10A9A00079FF00F01FF800F01DF800F01BF800F030
:10A9B00019F800F017F800F015F800F013F800F09F
:10A9C00011F8FFF767FFFFF765FFFFF763FFFFF77A
:10A9D00061FFFFF75FFFFFF75DFFFFF75BFFFFF72B
:10A9E00059FF00BD0C484021816100BF00BF00BF7E
:10A9F00000BF00BF00BF00BF00BF00BF00BF00BF5F
:10AA000000BF00BF00BF00BF816200BF00BF00BF2A
:10AA100000BF00BF704700000004005000B5FFF702
:10AA2000E1FFFFF7DFFFFFF7DDFFFFF7DBFFFFF7DA
:10AA3000D9FFFFF7D7FFFFF7D5FFFFF7D3FFFFF7EA
:10AA4000D1FFFFF7CFFFFFF7CDFFFFF7CBFFFFF7FA
:10AA5000C9FFFFF7C7FFFFF7C5FFFFF7C3FFFFF70A
:10AA6000C1FFFFF7BFFFFFF7BDFFFFF7BBFFFFF71A
:10AA7000B9FFFFF7B7FFFFF7B5FFFFF7B3FF00BD63
:10AA800008B5002808D00246002106480091044B72
:10AA90000068FEF7B9FB08BD002000F005F808BD0E
:10AAA000A9AA0008D4000020044972B60248C86070
:10AAB000BFF34F8F704700000400FA0500ED00E07F
:10AAC00010B5144812490180134981801349C1808F
:10AAD0000A2303810021418181810122C281818376
:10AAE0004324C486022404870D4C44878287C2878E
:10AAF00002464032118451849184C1839180142490
:10AB000084821182E12109018184038410BD000047
:10AB1000AA5500007406002034120000102700001F
:10AB20003C0F00000088704770470000F8B50446ED
:10AB300000206A461080194D55222A70AA226A7098
:10AB40000322AA70661DEE702A716971144A4900C9
:10AB50008918AC712246E81DFAF710FB002007E0C7
:10AB600029186A468978128889186A461180401C1B
:10AB7000B042F5DB611DA81CFBF7A4FA014668464C
:10AB8000018029190078C871684640780872224609
:10AB900009320249002001F01FFBF8BDD80A00204D
:10ABA00074060020F8B5164604460F46012205201B
:10ABB0001D46D1030007FCF788FAFFF70BFE384665
:10ABC000FFF714FE3046FFF711FE2846FFF70EFE92
:10ABD0002046FFF70BFEFFF7FDFDF8BD10B5012184
:10ABE00005200022C9030007FCF76FFA10BD000022
:10ABF00010B5FBF721FAFEF725FA00280DD0FEF775
:10AC000021FA0B24E40100190069002805D0FEF7A1
:10AC100019FA0019016902A08847002010BD000040
:10AC20004F4B0D0A0000000010B5FBF723FAFEF7AA
:10AC300009FA00280DD0FEF705FA0B24E4010019EB
:10AC40000069002805D0FEF7FDF90019016902A08E
:10AC50008847002010BD00004F4B0D0A0000000087
:10AC600010B5022814DAFEF7EDF900280DD0FEF732
:10AC7000E9F90B24E40100190069002805D0FEF76A
:10AC8000E1F90019016907A088470020C04310BD01
:10AC90004868FAF7BFFA002801D1FEF737F800201C
:10ACA00010BD000064656275675F6F666620666C44
:10ACB00061670D0A0000000010B5022814DAFEF7E3
:10ACC000C1F900280DD0FEF7BDF90B24E4010019ED
:10ACD0000069002805D0FEF7B5F90019016907A041
:10ACE00088470020C04310BD4868FAF793FA00284F
:10ACF00001D1FEF711F8002010BD000064656275F7
:10AD0000675F6F6E20666C61670D0A0010B5FFF714
:10AD10005FFBFEF797F900280DD0FEF793F90B249F
:10AD2000E40100190069002805D0FEF78BF900192D
:10AD3000016902A08847002010BD00004F4B0D0A9A
:10AD40000000000010B5FFF74FFBFEF77BF900286D
:10AD50000DD0FEF777F90B24E401001900690028F3
:10AD600005D0FEF76FF90019016902A0884700209D
:10AD700010BD00004F4B0D0A0000000070B5FEF73B
:10AD800061F90B25ED0100280CD0FEF75BF94019A5
:10AD90000069002806D0FEF755F9401902690FA195
:10ADA00011A09047FEF74EF9002815D0FEF74AF99A
:10ADB0004019006900280FD0FBF7D4F8FAF7EAFC35
:10ADC00004460E46FEF73EF9401905690B48224637
:10ADD000017833460AA0A847002070BD76312E3096
:10ADE0002E302E340000000056657273696F6E3A83
:10ADF00020202020202025730D0A0000380000208C
:10AE0000426174746572793A2020202020202575D3
:10AE1000252520252E3266560D0A000010B5112179
:10AE20000248FEF7D9F8002010BD0000E4D1000868
:10AE30000020704710B5072814D0FEF703F900284A
:10AE40000DD0FEF7FFF80B24E4010019006900287B
:10AE500005D0FEF7F7F80019016903A08847002024
:10AE6000C04310BD002010BD75736167653A207244
:10AE700074635F7365742079797979206D6D2064CE
:10AE800064206868206D6D2073730D0A0000000057
:10AE900010B50020FFF7F4FD002010BD10B50B2405
:10AEA000E401062812DAFEF7CDF800280BD0FEF7F1
:10AEB000C9F800190069002805D0FEF7C3F8001989
:10AEC00001690BA088470020C04310BDFEF7BAF807
:10AED00000280BD0FEF7B6F800190069002805D04D
:10AEE000FEF7B0F80019016911A08847002010BDD5
:10AEF0007365745F616463206E6F726D616C5F6D0A
:10AF0000696E206E6F726D616C5F6D617820657225
:10AF1000726F725F6D696E206572726F725F6D61C4
:10AF200078206572726F725F636E740D0A000000A4
:10AF30004F4B0D0A0000000010B50B24E40102285D
:10AF40000FDAFEF77FF800281BD0FEF77BF8001918
:10AF50000069002815D0FEF775F8001901690AA0EC
:10AF60000EE0FEF76FF800280BD0FEF76BF8001923
:10AF70000069002805D0FEF765F80019016904A0F2
:10AF80008847002010BD00004552524F520D0A0064
:10AF90004F4B0D0A0000000070B500250B24ED4357
:10AFA000E40102280FDAFEF74DF8002822D0FEF760
:10AFB00049F80019006900281CD0FEF743F8001971
:10AFC000016916A015E04868FAF724F9002801D0B5
:10AFD000082811D9FEF736F800280BD0FEF732F812
:10AFE00000190069002805D0FEF72CF80019016946
:10AFF0000EA08847284670BDFEF724F800280BD025
:10B00000FEF720F800190069002805D0FEF71AF8AD
:10B010000019016908A08847002070BD7365745F3E
:10B020006465765F69642069640D0A00696420655F
:10B0300072726F720D0A00004F4B0D0A0000000083
:10B0400010B50B24E401032812DAFDF7FBFF0028FA
:10B050000BD0FDF7F7FF00190069002805D0FDF7B8
:10B06000F1FF001901690BA088470020C04310BD03
:10B07000FDF7E8FF00280BD0FDF7E4FF0019006999
:10B08000002805D0FDF7DEFF001901690AA08847F6
:10B09000002010BD7365745F6970205B7365727604
:10B0A00065725F69705D205B7365727665725F7053
:10B0B0006F72745D0D0A00004F4B0D0A0000000016
:10B0C00010B50B24E401032812DAFDF7BBFF0028BA
:10B0D0000BD0FDF7B7FF00190069002805D0FDF778
:10B0E000B1FF001901690BA088470020C04310BDC3
:10B0F000FDF7A8FF00280BD0FDF7A4FF0019006999
:10B10000002805D0FDF79EFF001901690AA08847B5
:10B11000002010BD7365745F77696669205B737387
:10B1200069645D205B70617373776F72645D205B2F
:10B1300069705D0D0A0000004F4B0D0A0000000011
:10B1400010B5FFF765F9002010BD10B5FEF7EEFE53
:10B15000002010BD10B5FEF783F8FBF7D1FF10BD3E
:10B1600010B59AB034216846FAF721F8142115A8D1
:10B17000FAF71DF820210DA8FAF719F823480168FD
:10B180000324E402A143C21489180160FCF79EF96C
:10B190001F480169214301610E200090FF2001300A
:10B1A00002901020049002200990400401210B908D
:10B1B0000001059100240C9003910A946846FCF765
:10B1C000F9FB002801D072B6FEE70F20159003208E
:10B1D0001690179418940121199415A8FCF77CFA7D
:10B1E000002801D072B6FEE787200D9003200F944F
:10B1F00080041490109411940DA8FCF7A3F9002872
:10B2000001D072B6FEE71AB010BD00000070004019
:10B210004010024002490148886070470050000811
:10B2200000ED00E0F0B402680124A407144D154EAF
:10B23000154FA04205D0A84203D0B04201D0B84279
:10B2400003D170239A434B681A43A04205D0A84209
:10B2500003D0B04201D0B84204D103231B029A4369
:10B26000CB681A4380239A430B691A4302608A68A9
:10B27000C2620968816201214161F0BC704700002F
:10B2800000040040000801400014014010B4C90649
:10B29000C90E01238B40046A9C430462036A8A40FE
:10B2A0001343036210BC704730B48468FF252D023D
:10B2B000AC431B0213430B432343836030BC7047F2
:10B2C000826870239A430A4307210A4382607047C9
:10B2D00030B4026A520852000262026A446883690A
:10B2E0007025AB439B089B000D681D4302239A43C6
:10B2F0008B6813434460856149684163036230BCD5
:10B30000704730B4026A10239A430262036A4568A8
:10B31000826907242403A24303242402A2430C6865
:10B3200024021443202293438A6812011A43456081
:10B33000846149688163026230BC704730B4026A3C
:10B34000FF2301339A430262026A4468C36970258D
:10B35000AB439D08AD000B682B4301256D02AA434A
:10B360008D682D0215434460C3614968C16305625D
:10B3700030BC704730B4026A01231B039A43026257
:10B38000036A4568C26907242403A24303242402F4
:10B39000A2430C68240214430122520393438A6897
:10B3A00012031A434560C46149680164026230BCFB
:10B3B000704730B4036A046A6408640004628469F4
:10B3C000F025AC43120122430A24A3430B438261BC
:10B3D000036230BC704730B4036A1024A343036295
:10B3E0008369046A0F252D03AB4312031A43A0237C
:10B3F0009C43090121438261016230BC7047000017
:10B4000010B505480549806A884204D3642001F0DC
:10B41000F0FC01F05DF810BD00000020002F0D00D1
:10B4200010B4818CC90707D001684A6801235B0406
:10B430009A43836A1A434A60818C890707D5016859
:10B440004A6801231B049A43C36A1A434A60818CE9
:10B45000490707D501684A6801239B049A43036B97
:10B460001A434A60818C090707D501684A6801239D
:10B47000DB039A43436B1A434A60818CC90607D5A4
:10B4800001688A6801231B039A43836B1A438A600D
:10B49000818C890607D501688A6801235B039A437A
:10B4A000C36B1A438A60818C490612D501684B68C8
:10B4B00001221205046C934323434B60016C9142BB
:10B4C00007D101684A6803235B059A43436C1A431A
:10B4D0004A60818C090607D501684A680123DB04AC
:10B4E000806C9A4302434A6010BC7047F0B583B049
:10B4F00004462646002780367760FBF7EDFD029074
:10B500002068006825460007603500281CDA2A48B4
:10B5100000900121002249052046029B00F09AFC80
:10B52000002811D0EFF31081012080F310882068EB
:10B53000026880239A43026081F310882020E0672C
:10B540002F76032003B0F0BD20680068400729D59E
:10B55000194800900121002289052046029B00F035
:10B5600079FC00281ED0EFF31081012080F31088B1
:10B5700020680268FF2321339A43026081F3108818
:10B58000EFF31081012080F3108820688268520850
:10B590005200826081F31088202030602F760320D3
:10B5A00003B0F0BD2020E0673060276667662F7625
:10B5B000002003B0F0BD0000FFFFFF0110B5806A5E
:10B5C0000022014640314A834A82FCF7DFFF10BD6A
:10B5D000F8B5846AE06F254680352E682168896851
:10B5E00000270906002906DA212804D15220075332
:10B5F000204600F0DFF820688068400606D5222E3D
:10B6000004D15A200753204600F090F868681021B2
:10B61000084368602046FCF7B9FFF8BD70B50146E5
:10B62000886A0968096800238906002937DB5A21DE
:10B630000B52EFF31082012181F3108801680C682E
:10B64000FF250135AC430C6082F31088EFF31082C4
:10B65000012181F3108801688C68640864008C60A3
:10B6600082F31088EFF31082012181F310880168C2
:10B670008C684025AC438C6082F3108820228021A6
:10B680000A50016E01290AD1EFF3108281F310886C
:10B6900001680C681025AC430C6082F31088436687
:10B6A000016E012902D0FDF717FA70BD5821095A21
:10B6B000FCF748FF70BD10B5806A01214166016E3C
:10B6C000012902D0FDF70CFA10BD5821095A49088A
:10B6D000FCF738FF10BD10B50146886A0968096893
:10B6E00089061BD4002252210A52EFF31082012155
:10B6F00081F3108801688B688024A3438B6082F3F8
:10B700001088EFF31081012282F31088006802682C
:10B7100040231A43026081F3108810BDFDF7F0FA50
:10B7200010BD10B5806AFDF7EFFA10BD10B4EFF34D
:10B730001082012181F3108801680B68FF242134F5
:10B74000A3430B6082F31088EFF31082012181F391
:10B75000108801688B685B085B008B6082F310883F
:10B76000016E01290AD1EFF3108281F3108801687C
:10B770000B681024A3430B6082F3108820228021E1
:10B780000A5000210166816610BC704710B5EFF3C6
:10B790001082012181F3108801680B684024A343C3
:10B7A0000B6082F310882021C1670021C166FDF77C
:10B7B000A7FA10BD10B4EFF31082012181F31088B5
:10B7C00001680B68C024A3430B6082F3108820211A
:10B7D000C16710BC7047000070B5014640318B8BCB
:10B7E00002468032156814460268222D04D0906902
:10B7F00008210843906170BD526A456D1A402A8045
:10B80000426D921C42654A8B521E4A834A8B002A23
:10B81000F1D1EFF31083012282F3108802681568DA
:10B82000FF262136B543156083F31088EFF31083AC
:10B83000012282F31088026895686D086D0095609A
:10B8400083F3108820222260002484664466184B0B
:10B8500002689A420ED053681B020BD5EFF3108397
:10B86000012585F3108815680126B606B5431560D5
:10B8700083F31088026E012A02D0FDF72DF970BD06
:10B880000466EFF31083012282F3108802681568C2
:10B890001024A543156083F310880268D369DB4345
:10B8A000DB0600D41462098BFCF74CFE70BD00006F
:10B8B0000048004070B5014640318B8B0246803213
:10B8C000156814460268222D04D0906908210843A7
:10B8D000906170BD526A1A40436D1A70426D521CDD
:10B8E00042654A8B521E4A834A8B002AF1D1EFF3FC
:10B8F0001083012282F3108802681568FF26213622
:10B90000B543156083F31088EFF31083012282F3AF
:10B910001088026895686D086D00956083F3108843
:10B9200020222260002484664466184B02689A42F2
:10B930000ED053681B020BD5EFF31083012585F35E
:10B94000108815680126B606B543156083F3108884
:10B95000026E012A02D0FDF7BFF870BD0466EFF356
:10B960001083012282F31088026815681024A54311
:10B97000156083F310880268D369DB43DB0600D4CB
:10B980001462098BFCF7DEFD70BD0000004800402A
:10B99000F8B504460025904F20682269A168E36944
:10B9A000114362691A43114302688C4B1A400A43DF
:10B9B000026020684168032212039143E268114348
:10B9C0004160A0692168B94201D0226A10438A68A7
:10B9D0000B231B029A4302438A60814922688148F3
:10B9E0008A4213D1C0688007800F07D0012809D090
:10B9F000022805D0032807D0102142E0012140E0B1
:10BA000002213EE004213CE008213AE076498A42E6
:10BA100013D1C0680C21084007D0042809D0082899
:10BA200005D00C2807D010212BE0002129E00221AD
:10BA300027E0042125E0082123E06C498A4201D156
:10BA400000211EE06A498A4201D1002119E0BA4270
:10BA500016D1C0680321890208400BD00121890258
:10BA6000401A0BD0401A07D0884201D1082108E0C3
:10BA7000102106E0002104E0022102E0042100E0A0
:10BA800010215D485B4E8300BA4236D1002913D0A5
:10BA9000022914D0042917D0082918D00020012524
:10BAA000002861D0626851005118814202D8110308
:10BAB00081420FD2012589E0FBF712FFF0E73168E0
:10BAC000C906EDD41846EBE7FBF72AFFE8E70120AB
:10BAD000C003E5E7010E0602500800233018594163
:10BAE000F9F71CFB03210902444A411A914202D88A
:10BAF0002168C8606AE0012568E00122E769D20395
:10BB0000974234D1092919D20F007F443F79FF1998
:10BB1000BF4404070A140F1414141200FBF7E0FECC
:10BB20000EE0FBF7EDFE0BE03168C90608D41846BD
:10BB300006E0FBF7F5FE03E0104601E000200125DA
:10BB4000002843D0616840004A088018F9F7D0FA0D
:10BB500002462B49103A8A4207D8491C0140000787
:10BB6000420F0A432068C26030E001252EE0092917
:10BB700019D20F007F443F79FF19BF4404070A140C
:10BB80000F1414141200FBF7ABFE0EE0FBF7B8FE27
:10BB90000BE03168C90608D4184606E0FBF7C0FE82
:10BBA00003E0104601E00020012500280ED0616866
:10BBB0004A081018F9F79CFA0146114A10399142C7
:10BBC00003D8216880B2C86000E001250020A0668B
:10BBD000E0662846F8BD000000480040F369FFEF2A
:10BBE000003801404010024000440040004C00403A
:10BBF000005000400010024000093D00FFFC0F0013
:10BC0000EFFF000070B50446616558200253002123
:10BC100025468035696022202860606F002819D091
:10BC2000214BC362636F21481863636F20485863D8
:10BC3000606F81632168666D134624313246606F00
:10BC4000FBF711F8002805D010206860202028603C
:10BC5000012070BD206900280CD0EFF31081012075
:10BC600080F3108820680268FF2301331A430260C2
:10BC700081F31088EFF31081012080F31088206891
:10BC8000836801221343836081F31088EFF31081EE
:10BC900082F310882068826840231A43826081F30F
:10BCA0001088002070BD00001DB60008B7B600085F
:10BCB000D1B5000870B44165014640310A834A831A
:10BCC00000248466012382681B03FF259A4207D162
:10BCD0000269002A01D08D8319E02B4A8A8316E07D
:10BCE0007F26002A09D001252D07AA420ED102691C
:10BCF000002A09D03F228A8309E00269002A01D084
:10BD00008E8304E08D8302E08E8300E08C83014605
:10BD100080314C6022220A60EFF31082012181F30E
:10BD2000108801688C6801252C438C6082F3108890
:10BD30008168994202D10169002912D013498166B4
:10BD40000169002910D0EFF31081012282F31088DD
:10BD500000680268FF2321331A43026081F31088D0
:10BD60000EE00B498166EBE7EFF31081012282F3CD
:10BD700010880068026820231A43026081F310884B
:10BD800070BC002070470000FF010000B5B800083B
:10BD9000D9B7000810B4C16F212910D10146403134
:10BDA0004A8A002A0DD0C26C03681288D205D20DCF
:10BDB0009A62C26C921CC264488A401E488210BCBF
:10BDC0007047EFF31082012181F3108801680B683E
:10BDD0008024A3430B6082F31088EFF310810122CB
:10BDE00082F310880068026840231A43026081F3DE
:10BDF000108810BC704710B4C16F21290ED10146C4
:10BE000040314A8A002A0BD0C26C036812789A62C9
:10BE1000C26C521CC264488A401E488210BC7047E3
:10BE2000EFF31082012181F3108801680B688024F0
:10BE3000A3430B6082F31088EFF31081012282F399
:10BE400010880068026840231A43026081F310885A
:10BE500010BC7047FFB583B00C9D04460E461746D4
:10BE60002068C1693046884327D00020B84245D1B8
:10BE700020468030029020380190681C36D0FBF7B5
:10BE80002BF90699401AA84219D8002D17D020681E
:10BE9000016849072AD5C169C943090712D4206836
:10BEA000082505622046FFF741FC0298456001998C
:10BEB00000200876012007B0F0BD0120D6E703205E
:10BEC00007B0F0BDC069C04300050FD40120216850
:10BED000C00208622046FFF729FC02982021416039
:10BEE000019900200876032007B0F0BD2068C169E1
:10BEF0003046884305D00020B842BED0002007B0AD
:10BF0000F0BD0120F8E7000010B50248FCF742FB45
:10BF100010BD0000CC04002010B50248FCF73AFB2D
:10BF200010BD000054050020F8B51D4D0E0034D0A2
:10BF3000032832D2742148431A494418A0780028B3
:10BF400002D0012822D028E0E168A0684218606889
:10BF50000090406F006840682769101A0818C01BDD
:10BF6000F9F7C6F8012905D817D100980068C0690B
:10BF7000800612D43878307061692069884201D116
:10BF8000A06800E0401C2061002506E02046183033
:10BF90003146FCF707FF0028F6D02846F8BD000020
:10BFA000FFFFFFFF2C28002070B50C00064601D0D3
:10BFB000032E02D30020C04370BD742148432149A1
:10BFC0000E54227845186A706078A8706068A8607E
:10BFD000A168E9606278002A02D0012A05D00BE04E
:10BFE00028614018401E686106E028461830012389
:10BFF000A2686168FCF7B1FEE068E8622069286326
:10C00000A0692867606968632078002801D001284A
:10C0100006D121460C310EC928463830FDF72FFBDA
:10C020006078002804D0012806D0022804D006E059
:10C03000304600F009F802E0304600F021F8002018
:10C0400070BD00002C28002038B50C4974225043E4
:10C0500042185068016804E04C6A6B461C801C88DA
:10C060001C80CB691B07F7D491681161D368CC1889
:10C07000641E54619AB2FCF7C7FC38BD2C2800201E
:10C0800074214843044910B540180146683140689E
:10C090000122FCF7EDFC10BD2C28002070B50546F0
:10C0A00074201A4968434418A078002802D0012857
:10C0B00007D00DE0A0682061E1684018401E606173
:10C0C00006E0204618300123E268A168FCF745FE2F
:10C0D0006078002801D0012806D121462C310EC9F4
:10C0E00020463830FDF7CBFAA078002804D001288C
:10C0F00006D0022804D006E02846FFF7A5FF02E09C
:10C100002846FFF7BDFF002070BD00002C2800204E
:10C1100070B50D0001D0032802D30020C04370BDCC
:10C12000742148430449441874212046FDF7C8F897
:10C130000020656070BD00002C28002010B502466C
:10C140000E490020742343435B185B6893420FD170
:10C150007422424351188978002906D0012901D060
:10C16000022901D1FFF78CFF10BDFFF76DFF10BD55
:10C17000401CC0B20328E5D310BD00002C280020CD
:10C1800038B50146134800247422624312185268DD
:10C190008A4219D1742161430818817801290BD092
:10C1A000022908D1016F002902D0806EC0B28847F1
:10C1B0002046FFF765FF38BD816E6A4611706946FB
:10C1C0001830FCF7AFFDF3E7641CE4B2032CDBD3BB
:10C1D00038BD00002C280020F7B582B00021009166
:10C1E00003991546002903D0002D01D0032803D35D
:10C1F0000020C04305B0F0BD742148432B494618C8
:10C20000707834463834002804D0012820D0022821
:10C2100042D049E0FCF7AAFE20462946FDF701FA84
:10C22000070033D020463946FDF7C7F92A4638685B
:10C230000399F8F7A3FF2046FDF7D5F90446FDF76B
:10C2400023F8A088216882B27068FCF7BBFC2BE061
:10C25000FCF78CFE20462946FDF7E3F9070015D0D0
:10C2600020463946FDF7A9F92A4638680399F8F7B8
:10C2700085FF2046FDF7B7F90446FDF705F8A088CD
:10C28000216882B27068FCF7F7FC0DE0FCF7FCFF58
:10C290000020C043009007E0134664204343AAB245
:10C2A00070680399FCF71DFC0098A3E72C28002078
:10C2B00070B51F4A002174234B439B185B6883426F
:10C2C00031D1742041438C186078002816D00128A1
:10C2D00013D1204638300546FDF785F9014628463A
:10C2E000FDF755F92846FDF77EF9002805D081882D
:10C2F0008AB201686068FCF7BFFC70BD2046383028
:10C300000546FDF770F901462846FDF740F9284635
:10C31000FDF769F90028F0D081888AB20168606869
:10C32000FCF750FC70BD491CC9B20329C3D370BDD2
:10C330002C280020F8B53E4C002321783D4A1D46AC
:10C34000082910D0072947D0062950D0052952D0F6
:10C35000042953D0032954D0002956D0012958D09C
:10C3600002295AD05BE0A17800264A1F04E0314F31
:10C37000BF5DFB189BB2761C9642F8DB6679277985
:10C380009A195118E3786278C9188918C9194018A0
:10C39000C0430006000E1AD1012E14D0022E16D171
:10C3A00025482449C018F8F7E9FE00F0F9FE64209A
:10C3B00000F01FFDBFF34F8F21492048C860BFF335
:10C3C0004F8F00BFFDE759081046FEF7AFFB257001
:10C3D000E570A570A571F8BDA1795054491CC8B28B
:10C3E000A071A178491F8842F5D1082001E0607052
:10C3F00007202070F8BDE0700620FAE76071052084
:10C40000F7E7A070E5700420F3E7552807D1012075
:10C41000EFE7AA2803D10220EBE7032803D0257019
:10C42000E570A570F8BD032020702071F8BD0000F4
:10C4300076000020740A0020740600200400FA052B
:10C4400000ED00E07CB51546024600201C460029A0
:10C450000BD0491E00920191044B6A4621462846A2
:10C4600000F020F9009A002111707CBDDDCD00089C
:10C470002021020C01D010211046020A01D01046E2
:10C480000839020901D01046091F820801D0104660
:10C49000891E420801D0881E7047081A7047F0B400
:10C4A000040C8BB2264682B25E430D0C1046370C4C
:10C4B0005843360480190021794116466E43370CE3
:10C4C00036048019794126466E438919F0BC7047BD
:10C4D000BFF34F8F04490348C860BFF34F8F00BFBD
:10C4E000FDE700000400FA0500ED00E0BFF34F8F08
:10C4F00004490348C860BFF34F8F00BFFDE7000049
:10C500000400FA0500ED00E000487047B403002085
:10C5100002E008C8121F08C1002AFAD1704770470C
:10C52000002001E001C1121F002AFBD1704700006A
:10C53000F0B51FB486B00998089A030D0021024394
:10C5400014D05148514A1818504305141198012825
:10C5500010981AD0281A401C00264D4F4D490096BD
:10C5600001910490002812DA444211E0119801244C
:10C5700049A3012801D11098C1430698119A8460FB
:10C580000360C26041600BB0F0BD4042E4E7044686
:10C59000210500203F4A001C51410391029012E006
:10C5A000E00707D032463B4601990098F8F7D2FFE2
:10C5B0000191009032463B4610461946F8F7CAFFF3
:10C5C00006460F466410002CEAD10498039B00280D
:10C5D000029A0999089806DAF8F7BCFF019B009ABD
:10C5E000F8F7B8FF05E0F9F71DF8019B009AF9F795
:10C5F00019F804460E460022284BF9F7DFF803D855
:10C600000020C043014607E00022254B204631466A
:10C61000F8F7EEFEF9F70EFA102409E0002C0ADB19
:10C620000A220023F8F77AFD079B30321A55641E60
:10C6300002460A43F2D11122641C079B121B1C19EB
:10C64000119B012B03D0012308430ED10AE00843BC
:10C6500004D0112010900020119077E71098151A3F
:10C660006D1E0BE01098824202DD00236D1C03E07A
:10C67000824201DA00236D1E002BEED0069811993C
:10C680008260C16030C07EE701FCFFFF104D0000FA
:10C69000000014400000F03F300000000000F043B4
:10C6A0000000E03FFFB597B00646002518E22528B8
:10C6B00077D100242746FD49049400E00443761C0A
:10C6C00032780120203A90400842F7D130782A2869
:10C6D0000ED00222307801463039092916D8049943
:10C6E0000A235943303940181443761C0490F1E76B
:10C6F000189802C804911890002904DA0120400318
:10C7000004434842049002200443761C30782E28CB
:10C7100014D1042004437078761C2A2809D1189873
:10C72000761C80C8189009E00A214F43303FC71992
:10C73000761C3078014630390929F5D930786C28D3
:10C7400010D006DC4C281AD068280ED06A2817D1E1
:10C7500004E0742813D07A2812D110E0012040059B
:10C7600004430CE00121090501E0032109050C4304
:10C770007178814203D1012000052418761C761CB3
:10C780003078119066280BD013DC58287DD009DC56
:10C7900000287BD04528F6D04628F4D047281AD167
:10C7A000A5E118E0632835D0642870D0652812D13F
:10C7B0009DE170286CD008DC6728F1D069287BD017
:10C7C0006E280DD06F2806D1BAE073282ED07528B8
:10C7D00071D0782859D01A9A199990476D1C7EE12A
:10C7E0006002400F022809D003280DD004281898B1
:10C7F00001680DD00D60001D189070E11898EA17BF
:10C8000001680D604A60F6E7189801680D80F2E74C
:10C810000D70F0E718986A4601781172001D1890A3
:10C820000020507202A80090012005E0189802C86C
:10C83000189000200091C04361070DD5002101E050
:10C840000199491C0191B94212DA8142F8DB009A40
:10C85000515C0029F4D10BE0002101E00199491C51
:10C8600001918142FADB019A0099895C0029F5D196
:10C87000019904981A9B471A21463846199A00F0E4
:10C8800097FA0199401945180BE04FE02CE113E0AD
:10C890004EE0009800990078491C00911A9A199965
:10C8A00090470198401E0190401CF2D12146384625
:10C8B0001A9B199A10E137E00A200021009001919B
:10C8C0006002410F022907D0189A01CA1892C217B4
:10C8D0009446032908D00AE01898C01DC108C90071
:10C8E00005C91891944607E000B2C217944604297E
:10C8F00002D140B2C1178C4600226146944506DA47
:10C900000A460021404291418C462D2102E021053A
:10C9100004D52B216A461173012103E0E10701D000
:10C920002021F7E7029155E00A200AE0102008E0F4
:10C93000102000900021042004430191082703E007
:10C9400008200021019100906002410F022907D0C8
:10C95000189A01CA189200229446032908D008E0C8
:10C960001898C01DC108C90005C91891944603E074
:10C9700080B2042900D1C0B200210291210729D53B
:10C980001199702906D0009A1021019B4A401A4340
:10C9900005D00EE040216A461173012108E061468E
:10C9A000014306D030216A46117311995173022157
:10C9B0000291009A0821019B4A401A430AD161461C
:10C9C000014301D1610705D530216A461173012168
:10C9D0007F1E02911199582904D035A10E910DA9FD
:10C9E0000D910DE037A1F9E76146019B009AF8F738
:10C9F00095FB0E9B8C469B5C0D9A521E0D921370FC
:10CA000061460143F0D10D9805A9081A2030019024
:10CA1000600703D501200004844300E0012701984A
:10CA2000874201DD381A00E000200199009041188A
:10CA3000029809180498401A0490E00306D421468D
:10CA40001A9B199A049800F0B3F94519002706E0DB
:10CA500003A81A9AC05D199990476D1C7F1C029813
:10CA60008742F5DBE0030CD521461A9B199A0498FE
:10CA700000F09EF9451904E01A9A30201999904760
:10CA80006D1C0099481E00900029F5DC08E00D9807
:10CA90000D990078491C0D911A9A199990476D1CAF
:10CAA0000199481E01900029F1DC63E10928010089
:10CAB0003031323334353637383961626364656614
:10CAC00000000000303132333435363738394142D6
:10CAD000434445460000000000F05AF94519761C11
:10CAE0003078002800D0E2E528461BB0F0BD600792
:10CAF00000D406271898C01DC108C90048680A68F4
:10CB00000831C30FDB071891190001D09CA108E080
:10CB1000210501D59BA104E0E10701D09AA100E025
:10CB20009AA1430011985B08109165280CD006DC8F
:10CB3000452809D046281DD0472841D141E0662824
:10CB400018D067283CD13CE00021112F01DB1120D7
:10CB500000E0781C0191009008A911A8FFF7E8FCFB
:10CB6000139905910021119A15927F1C1298019733
:10CB7000009150E00120C00703900120019008A916
:10CB8000009711A8FFF7D4FC139A1499059200227C
:10CB9000119B009212981593059A0192002901D0D9
:10CBA000104602E0791C40180190381A01D501980E
:10CBB00004E04042401E0090781C0190C01B02908F
:10CBC00043E0012F00DA01270021112F01DD1120A0
:10CBD00000E038460191009008A911A8FFF7A8FCD1
:10CBE00013990591119A00211298159200910197BD
:10CBF00021070CD40599B94201DB019900E00191AC
:10CC0000012904DD159A491E515C302906D0B8422D
:10CC100001DA011D05DA0121029115E00199491E91
:10CC2000EDE7002805DC0099411800910199091AE7
:10CC300003E0019A411C914200DD01910099401AE4
:10CC4000401C02900120C0070390200706D40299DF
:10CC50000198814202DB0020C04302900020694617
:10CC6000C87707AF012103980337C907884224D04A
:10CC7000022011902B201290039800280CDA4042D9
:10CC800003902D20129007E00A210398F8F730FA5C
:10CC900030317F1E039039701199481E1190002980
:10CCA000F2DC03980028EFD1791E129808703078D2
:10CCB000202108404530BF1E387006A8C01BC01D8B
:10CCC000039010980078002800D0012001994118A5
:10CCD0000298C0170918039809180498401A401EB2
:10CCE0000490E00306D421461A9B199A049800F098
:10CCF0005FF8451910980078002803D01A9A1999FE
:10CD000090476D1CE00324D521461A9B199A04987C
:10CD100000F04EF845191CE00098002807DB009948
:10CD20000598884203DD1598405C199901E019992E
:10CD300030201A9A904700986D1C401C0090029871
:10CD4000401E0290002804D11A9A2E20199990476B
:10CD50006D1C0199481E01900029DDDC05E0387842
:10CD60001A9A7F1C199990476D1C0399481E0390CD
:10CD70000029F4DC21461A9B199A0498ACE60000BD
:10CD80002D0000002B00000020000000000000002B
:10CD9000F8B5044600251E461746880404D405E06D
:10CDA00039462020B0476D1C641EF9D52846F8BDD1
:10CDB000FFB50446002581B01E46C80301D53027C3
:10CDC00000E02027880404D505E038460399B047E1
:10CDD0006D1C641EF9D5284605B0F0BD4A68002ACE
:10CDE00006D00A68531C0B6010704868401E4860EB
:10CDF00070477D2110B5C900484300F001F810BD0F
:10CE0000002140E000BF00BF00BF00BF00BF00BF67
:10CE100000BF00BF00BF00BF00BF00BF00BF00BF1A
:10CE200000BF00BF00BF00BF00BF00BF00BF00BF0A
:10CE300000BF00BF00BF00BF00BF00BF00BF00BFFA
:10CE400000BF00BF00BF00BF00BF00BF00BF00BFEA
:10CE500000BF00BF00BF00BF00BF00BF00BF00BFDA
:10CE600000BF00BF00BF00BF00BF00BF00BF00BFCA
:10CE700000BF00BF00BF00BF00BF00BF00BF00BFBA
:10CE800000BF00BF491C8142BCD37047FAF740F98C
:10CE9000FEF766F9FDF72EF9FDF7F4F8FDF7CCF98A
:10CEA000FDF75CFAFDF776FAFDF7E2F9FDF706FA11
:10CEB0001F481E49016000214160816001621D4AD6
:10CEC000416242618162FAF7F7F9002801D072B637
:10CED000FEE7FDF757FBF8F7BDFFF8F73BFFFDF75F
:10CEE0007DFEFDF775FAFF20000203461A46114643
:10CEF000FDF758FEFF24F5342046F9F7EDFEFF203C
:10CF0000000403461A461146FDF74CFE2046F9F789
:10CF1000E3FEFDF769FA0124074DF8F743FFAC7013
:10CF2000F9F752F8FEF76CFAF7E70000007C0040D2
:10CF300014040020FFFF00000000002010B504468C
:10CF4000FCF760FC4E20FCF72FFCFCF797FCE0B2EE
:10CF5000FCF72AFCFCF792FCFCF754FC4F20FCF792
:10CF600023FCFCF78BFC0020FCF7F0FB0446FCF7ED
:10CF700065FC204610BD70B50D460446FCF742FC2A
:10CF80004E20FCF711FCFCF779FCE0B2FCF70CFC3E
:10CF9000FCF774FC2846FCF707FCFCF76FFCFCF779
:10CFA0004DFC0A20FFF72CFF70BD000010B52421B6
:10CFB000002000F04DF81B48FFF722FF00210F2052
:10CFC00000F046F80521102000F042F8042111205D
:10CFD00000F03EF883217F2000F03AF869217F209D
:10CFE00000F036F8BD217F2000F032F80E480078BE
:10CFF000262804D1002240218C2000F019F80120BD
:10D0000000F02AF8094814210187282000F020F8B0
:10D010000A20FFF7F5FE012000F036F8012000F0AD
:10D0200043F810BD204E0000D800002074060020F8
:10D03000F8B517460E4605460024FFF77FFF394630
:10D04000B44331402143284600F002F80020F8BDE7
:10D0500010B5FFF790FF10BD10B500280AD00021D1
:10D060002720FFF7F5FF04211920FFF7F1FF8721A3
:10D07000162005E000211620FFF7EAFF0021192005
:10D08000FFF7E6FF10BD000010B5002801D0002218
:10D0900000E0802280211120FFF7CAFF0148FFF73E
:10D0A000AFFE10BDA086010010B5002811D00121EF
:10D0B0002F20FFF7CDFF62213020FFF7C9FF462167
:10D0C0003120FFF7C5FF32210846FFF7C1FFA2213B
:10D0D00000E022213320FFF7BBFF10BD0C480D4AB2
:10D0E0000188914210D1C18832290DD3C18E4329C4
:10D0F0000AD8818F012907D8C08F012804D8044895
:10D1000040308088012801D90120704700207047F5
:10D1100074060020AA55000010B50124A40221467F
:10D120001948F8F744F8224617491848F9F79CF8C7
:10D130001548174902888A4224D001801549818008
:10D140001549C1800A230381002141818181012287
:10D15000C28181834324C486022404870F4C448700
:10D160008287C28702464032118451849184C183F0
:10D170009180142484821182E12109018184038435
:10D1800000F00EF810BD00007406002000FC00083E
:10D19000AA55000034120000102700003C0F0000C8
:10D1A00070B5FFF79BFF002801D0012070BD72B65B
:10D1B0000124074DA40221462846F9F73BF8002830
:10D1C00004D0224603492846F9F7DAF862B670BD62
:10D1D00000FC000874060020002100E0491C814288
:10D1E000FCD37047B0D300084BB1000898D30008B7
:10D1F00091AE000870D300087DAD000854D300083C
:10D20000B9AC000828D3000861AC000888D3000836
:10D2100031AE000890D3000835AE000814D30008E2
:10D220009DAE000880D3000841B000081CD3000860
:10D2300099AF000848D30008C1B00008A0D3000887
:10D2400039AF000868D3000845AD000840D3000896
:10D250000DAD000860D3000829AC000834D30008E5
:10D26000F1AB000878D3000841B1000800000000CD
:10D270000000000001020304060708090304060871
:10D280000C10182030000000000102030400404090
:10D290004040404040404041414141414040404089
:10D2A00040404040404040404040404040400502F7
:10D2B0000202020202020202020202020202202012
:10D2C00020202020202020200202020202020290C0
:10D2D00090909090901010101010101010101010CE
:10D2E000101010101010101010020202020202881A
:10D2F000888888888808080808080808080808082E
:10D30000080808080808080808020202024000008D
:10D310008ED200087365745F616463007365745F27
:10D320006465765F6964000064656275675F6F6657
:10D3300066000000626565705F6F66660000000051
:10D340006770735F6F6666007365745F776966699F
:10D350000000000064656275675F6F6E000000008A
:10D36000626565705F6F6E006770735F6F6E00005F
:10D37000696E666F00000000736C656570000000E8
:10D380007365745F697000007274635F6765740031
:10D390007274635F736574007265626F6F7400000E
:10D3A0007365745F636F6E74726173740000000064
:10D3B00074657374000000002B2B2B0D000000001F
:10D3C00061742B6A6F696E3D6F7461612C31300D31
:10D3D0000000000061742B63683D636E3437302CAD
:10D3E000330D000061742B64723D350D00000000A8
:10D3F00061742B6170706575693D3532363937332C
:10D40000363936653637343834360D0061742B635F
:10D410006C6173733D610D0061742B6170706B659D
:10D42000793D326237653135313632386165643283
:10D430006136616266373135383830396366346653
:10D4400033630D0061742B6D6F64653D6D61630D19
:10D450000000000061742B6164723D6F66660D0010
:10D4600061742B7265626F6F740D000061742B73B1
:10D470006C6565703D6C696768742C302C6C6576E2
:10D48000656C2C6C6F770D0061742B646576657527
:10D49000693D3437333635343966303033312530F1
:10D4A00034780D00636C6561720000006C730000DD
:10D4B000D0D4000800000020B8030000645B00081E
:10D4C00030D50008B8030020E82C000020C5000873
:10D4D000014B43500112041250022580392F0913C9
:10D4E0000D11BA0C0F13B8D3140844D41B08C0088C
:10D4F0001A0C081A88041AF00C1A18081AE4081AE8
:10D50000D4041A540C1A6C041A6004410A252781A9
:10D510009204021D2032021AA45C139D8F1B08ACDA
:10D52000084B51906801FF01FF0172720100000079
:04000005080050C1DE
:00000001FF
